:020000040800F2
:100000003837002001010008F52A0008BF1F00084A
:10001000F12A0008AD06000875370008000000004E
:10002000000000000000000000000000712F000828
:10003000FD06000800000000872C0008C92F0008FA
:100040001B0100081B0100081B010008192F0008F4
:100050001B0100081B0100081B0100081B01000810
:100060001B0100081B0100081B0100081B01000800
:100070001B0100081B0100081B0100081B010008F0
:10008000B1060008C10600081B0100081B0100089A
:100090001B0100081B0100081B0100081B010008D0
:1000A0001B0100081B0100081B0100081B010008C0
:1000B0002D300008B1300008153100081B01000880
:1000C0001B0100081B0100081B0100081B010008A0
:1000D0001B0100081B010008CD360008E1360008AE
:1000E0001B0100081B0100081B010008DFF80CD0F1
:1000F00000F09CF9004800471568000838370020D8
:100100000648804706480047FEE7FEE7FEE7FEE7B1
:10011000FEE7FEE7FEE7FEE7FEE7FEE7D52F000875
:10012000ED000008202A04DB203A21FA02F0002129
:10013000704721FA02F3D040C2F1200291400843F7
:100140001946704710B540EA01040346A40703D0DE
:1001500009E010C9121F10C3042AFAD203E011F8F3
:10016000014B03F8014B521EF9D210BDD2B201E08F
:1001700000F8012B491EFBD270470022F6E710B5AC
:1001800013460A4604461946FFF7F0FF204610BD05
:1001900030B505462A460B4612F8010B13F8014B01
:1001A00008B1A042F8D01CB1002802D06D1CF1E7C4
:1001B000284630BD10B5044604E00B7800F8013B3A
:1001C00003B1491C521EF8D2204610BDCAB2401ECF
:1001D00010F8011F8A4202D00029F9D1002070478F
:1001E000421C10F8011B0029FBD1801A704710B582
:1001F000002200E0521C835C8C5CA34201D1002BE6
:10020000F8D1D8B2E1B2401A10BD30B50446002092
:10021000034600E05B1C934203D2E05CCD5C401BD4
:10022000F8D030BD034611F8012B00F8012B002A4D
:10023000F9D11846704730B505460020034600E066
:100240005B1C934205D2EC5CC85C201A01D1002CE7
:10025000F6D130BD70B5064603F03CFB0468054698
:100260000A220021304600F04CF82C6070BD70B5B9
:10027000064603F02FFB046805460A22002130469B
:1002800000F03FF82C6070BD0EB540F23342029290
:100290000022CDE90022134600F07AF803B000BD39
:1002A0002DE9F05F0546002092469B4688460646AB
:1002B000814640241BE02846414647462246FFF738
:1002C00031FF53465A46C01A914110D31146184681
:1002D000224600F0BDF82D1A67EB01084F46224672
:1002E0000120002100F0B4F817EB00094E41201E58
:1002F000A4F10104DFDC484631462A464346BDE806
:10030000F09F2DE9F04791460F46804604460026AF
:1003100014F8015B2DB100F0ABF80068405DC00738
:10032000F6D12B2D02D02D2D18D0641E4A46394609
:10033000204600F0A1F827B13968A14201D1C7F8E1
:10034000008071054FF002040BD54042002803DD08
:1003500003F0C0FA0460A007BDE8F08746F48066A9
:10036000E4E70028F8DA03F0B5FA04606FF0004023
:10037000F2E710B5141E73F1000408DA401C41F1D5
:10038000000192185B411A4301D120F0010010BD19
:100390002DE9F04D92469B4611B1B1FA81F202E08F
:1003A000B0FA80F22032904600F052F804460F4630
:1003B00040EA0A0041EA0B0153465A46084313D06B
:1003C000114653EA010019D0C8F140025046FFF728
:1003D000A9FE05460E4650465946424600F038F8FA
:1003E000084305D0012004E020463946BDE8F08DE1
:1003F0000020054346EAE0762C4337430A9863051C
:10040000E40AA0EB08000022FD0A44EA47540A303F
:1004100002D500200146E9E7010510196941DDE92F
:10042000084500196941BDE8F04DA2E7064C074DAB
:1004300006E0E06840F0010394E8070098471034B4
:10044000AC42F6D3FFF756FED4AA0008F4AA00087F
:10045000202A04DB203A00FA02F100207047914084
:10046000C2F1200320FA03F31943904070470000C3
:100470000048704730A700082DE9F05F82460078F9
:10048000002715468B460AF10104B946302801D0F1
:100490009DB113E014F8010B0127782803D05828E8
:1004A00001D045B10AE00DB1102D07D1002710256C
:1004B00014F8010B02E0082500E00A250026B046EA
:1004C0000EE005FB080005FB06F1012701EB1046D5
:1004D0001FFA80F8B6F5803F00D3B94614F8010B37
:1004E000294600F018F80028EBDABBF1000F05D020
:1004F0000FB1641E00E05446CBF80040B9F1000F84
:1005000006D003F0E7F902210160C81EBDE8F09FA4
:1005100048EA0640FAE73A2800D2303820F02002B4
:10052000412A01D3A2F13700884201D34FF0FF30B6
:10053000704770B58C1810F8015B15F0070301D1F6
:1005400010F8013B2A1106D110F8012B03E010F836
:10055000016B01F8016B5B1EF9D12B0705D4002359
:10056000521E0DD401F8013BFAE710F8013BCB1AFB
:10057000921C03E013F8015B01F8015B521EF9D5F0
:10058000A142D8D3002070BD10B5FF2000F028F89C
:100590000446552C01D1002010BD5521FF2000F04C
:1005A0005DF8FF2000F01CF80446552C01D1002016
:1005B000F2E70120F0E710B501F02CFD10BD70B599
:1005C00006460C46154608E03046721C96B200F00E
:1005D00007F804F8010B681E85B2002DF4D170BD38
:1005E00070B50446002601F0F5FD2546E11704EB41
:1005F00011610912A02202EB4101C8B201F0B6FD5F
:1006000001F034FEE11704EB11610912A4EB0121A2
:10061000C8B201F0ABFD01F029FE01F0DBFDA12025
:1006200001F0A4FD01F022FE002001F067FD064666
:1006300001F0F6FD304670BD70B505460C46164615
:1006400006E02178284600F009F8681C85B2641C91
:10065000301EA6F101018EB2F3D170BD70B5044613
:100660000E4601F0B7FD2546E11704EB11610912B2
:10067000A02202EB4101C8B201F078FD01F0F6FDC5
:10068000E11704EB11610912A4EB0121C8B201F0DA
:100690006DFD01F0EBFD304601F068FD01F0E6FD77
:1006A00001F0BEFD0A2004F05DFB70BD00BFFEE757
:1006B00010B5024800F030F910BD000040050020E0
:1006C00010B5024800F028F910BD0000FC0400201D
:1006D00030B590F840500124AC40C56B6C600468A4
:1006E00063604468102C04D10468A2600468E1606F
:1006F00003E00468A1600468E26030BD704770B533
:1007000004460D461646204600F061F810B14FF041
:10071000FF3070BDD4F8CC0500EB400004EB0011B5
:100720002846FFF77FFDD4F8CC0500EB400204F526
:10073000F07000EB42113046FFF774FDD4F8CC05A1
:10074000401C0A21B0FBF1F201FB1200C4F8CC05F9
:10075000D4F8D005401EC4F8D0050120D9E7002107
:10076000C0F8C815C0F8CC15C0F8D015704770B5E2
:1007700004460E461546204600F032F810B14FF000
:10078000FF3070BDD4F8C81501EB410104EB011036
:100790003146FFF747FDD4F8C81501EB410204F5D7
:1007A000F07101EB42102946FFF73CFDD4F8C80573
:1007B000401C0A21B0FBF1F201FB1200C4F8C8058D
:1007C000D4F8D005401CC4F8D0050120D9E7014673
:1007D000D1F8D00508B9012070470020FCE70000DF
:1007E00010B50446012003F043F8962004F0C6FA41
:1007F0000A2209A0D4F8D01503F048F8962004F096
:10080000BDFA002003F034F8D4F8D0050A2801D14D
:10081000012010BD0020FCE76669666F20757365D6
:10082000643A25642F25640A000000000146002078
:100830000A68126822F00E020B681A600A681268D1
:1008400022F001020B681A6091F8403001229A40B0
:10085000CB6B5A60012281F8212000BF002281F871
:10086000202000BF7047000070B50446002594F8B2
:100870002100022803D00420A063012548E020685D
:10088000006820F00E00216808602068006820F0F1
:100890000100216808601F492068884201D10120B9
:1008A00026E01C4914312068884201D110201FE045
:1008B000184928312068884201D1801518E015496F
:1008C0003C312068884201D1801411E01149503137
:1008D0002068884202D14FF4803009E00D4964312C
:1008E0002068884202D14FF4801001E04FF0807000
:1008F000084908394860012084F8210000BF002021
:1009000084F8200000BF606B10B12046616B8847FF
:10091000284670BD0800024070B50446E06B0568CB
:100920002068066894F84010042088402840002879
:1009300046D006F00400002842D02068006800F08D
:10094000200028B92068006820F0040021680860B1
:1009500057492068884201D1042027E054491431C6
:100960002068884201D1402020E051492831206888
:10097000884201D1001519E04D493C312068884278
:1009800002D14FF4804011E049495031206888423B
:1009900002D14FF4802009E0454964312068884243
:1009A00002D14FF4800001E04FF0806040490839E7
:1009B0004860E06A00287AD02046E16A884776E0FD
:1009C00094F84010022088402840A0B306F00200AE
:1009D00088B32068006800F0200040B920680068F3
:1009E00020F00A0021680860012084F821003049C5
:1009F0002068884201D1022028E02D491431206866
:100A0000884201D1202021E02949283120688842EC
:100A100001D140151AE026493C312068884202D1B4
:100A20004FF4005012E0224950312068884203D12F
:100A30004FF400300AE017E01D4964312068884215
:100A400002D14FF4001001E04FF00070184908394E
:100A5000486000BF002084F8200000BFA06A30B3C7
:100A60002046A16A884722E094F840100820884078
:100A70002840E0B106F00800C8B12068006820F006
:100A80000E002168086094F8401001208840E16B56
:100A900048600120A06384F8210000BF002084F892
:100AA000200000BF206B10B12046216B884770BD2D
:100AB000080002400146002209B901207047184B86
:100AC0000868C01A1423B0FBF3F0800008641448CF
:100AD0000838C863022081F821000868026843F6DC
:100AE000F0708243D1E901031843CB6818430B69C6
:100AF00018434B6918438B691843CB691843024369
:100B00000868026000208862C862086348638863DE
:100B1000012081F82100002081F8200000BFCDE7EE
:100B2000080002402DE9F04104460D4616461F46D6
:100B30004FF0000800BF94F82000012802D10220E5
:100B4000BDE8F081012084F8200000BF94F8210066
:100B500001282CD1022084F821000020A063206805
:100B6000006820F00100216808603B4632462946B3
:100B70002046FFF7ADFDE06A30B12068006840F024
:100B80000E00216808600BE02068006820F0040077
:100B9000216808602068006840F00A002168086049
:100BA0002068006840F001002168086006E000BF8E
:100BB000002084F8200000BF4FF002084046BFE745
:100BC0002DE9F8470346002400200025844600272D
:100BD00000226EE14FF0010808FA02F4D1F800801B
:100BE00008EA0400A0427DD1DFF8D0A2D1F8048049
:100BF000A8EB0A09D0453AD014DCB8F1030F50D065
:100C000009DCB8F1000F31D0B8F1010F1CD0B8F1F8
:100C1000020F49D120E0B8F1110F18D0B8F1120F2E
:100C200042D11EE0B9F5881F25D006DCB9F5803F1A
:100C300020D0B9F5801F37D11AE0B9F5001F18D0C0
:100C4000B9F5041F30D117E0D1F80CC02DE0D1F870
:100C50000C8008F1040C28E0D1F80C8008F1080C95
:100C600023E0D1F80C8008F10C0C1EE000BF00BF9F
:100C700000BF00BF00BF00BFD1F80880B8F1000F6F
:100C800002D14FF0040C0BE0D1F80880B8F1010F4D
:100C900003D14FF0080C1C6102E04FF0080C5C61BE
:100CA00003E04FF0000C00E000BF00BFFF2801D8B8
:100CB000984601E003F104084646FF2802D84FEAAF
:100CC000820803E0A2F108084FEA88084746D6F8F0
:100CD00000804FF00F0909FA07F928EA09080CFA11
:100CE00007F900E088E048EA0908C6F80080D1F872
:100CF000048008F08058B8F1805F7DD100BFDFF834
:100D0000C081D8F8188048F00108DFF8B491C9F81C
:100D10001880C846D8F8188008F00108CDF800807F
:100D200000BF00BF4FEAB9384FEA920958F829507E
:100D30004FEA82784FEA18794FF00F0808FA09F85D
:100D400025EA0805DFF87C81434502D14FF0000811
:100D500016E0DFF87481434502D14FF001080FE03F
:100D6000DFF86881434502D14FF0020808E0DFF860
:100D70006081434502D14FF0030801E04FF00408C1
:100D80004FEA82794FEA197908FA09F848EA050525
:100D9000DFF840814FEA920948F82950D1F80480E1
:100DA00008F48038B8F5803F0AD1DFF82C81D8F8F4
:100DB000008048EA0008DFF82091C9F8008009E0C7
:100DC000DFF81481D8F8008028EA0008DFF80891DD
:100DD000C9F80080D1F8048008F40038B8F5003F65
:100DE00010D1DFF8F48008F10408D8F8008048EA50
:100DF0000008DFF8E49000E05AE009F10409C9F8BE
:100E000000800DE0DFF8D08008F10408D8F80080F9
:100E100028EA0008DFF8C09009F10409C9F8008049
:100E2000D1F8048008F48018B8F5801F0ED1DFF8DF
:100E3000A88008F10808D8F8008048EA0008DFF820
:100E4000989009F10809C9F800800DE0DFF8888062
:100E500008F10808D8F8008028EA0008DFF8789040
:100E600009F10809C9F80080D1F8048008F40018D5
:100E7000B8F5001F0ED1DFF8608008F10C08D8F833
:100E8000008048EA0008DFF8509009F10C09C9F821
:100E900000800DE0DFF8408008F10C08D8F80080F1
:100EA00028EA0008DFF8309009F10C09C9F8008041
:100EB000521C102AFFF48EAEBDE8F8870000111016
:100EC0000010024000080140000C014000100140E9
:100ED0000014014008000140000401400AB1016112
:100EE00001E00B040361704701480068704700008F
:100EF00000000020034800680349097808440149BC
:100F000008607047000000200800002010B5084865
:100F1000006840F0100006490860032000F0C2F8A5
:100F2000002000F007F800F02BF8002010BD0000B2
:100F30000020024070B504460E4800784FF47A71E4
:100F4000B1FBF0F00C490968B1FBF0F5284600F060
:100F500034FC08B1012070BD102C07D200222146BC
:100F6000501E00F060F80548046001E00120F2E73F
:100F70000020F0E7080000206001002004000020AD
:100F800008B500BF1F48806940F001001D49886115
:100F90000846806900F00100009000BF00BF0320F8
:100FA00000F080F8002211466FF00B0000F03BF8D3
:100FB000002211466FF00A0000F035F800221146B9
:100FC0006FF0090000F02FF800221146501F00F0CA
:100FD0002AF800221146101F00F025F800221146C1
:100FE000901E00F020F800221146501E00F01BF861
:100FF00000BF0549486820F0E06040F0007048609C
:1010000000BF08BD001002400000014000BF00F01A
:101010001F02012191404209920002F1E022C2F830
:10102000001100BF70472DE9F05F80460D4616465F
:10103000002701F061FD074639462A46334601F094
:101040000700C0F1070ABAF1040F02D94FF0040AF1
:1010500001E0C0F1070AD14600F1040ABAF1070F16
:1010600002D24FF0000A01E0A0F1030AD4464FF08B
:10107000010A0AFA09FAAAF1010A0AEA020A0AFAB4
:101080000CFA4FF0010B0BFA0CFBABF1010B0BEA66
:10109000030B4AEA0B042146404601F035FDBDE84A
:1010A000F09F000000BF00F00702064B19684FF6E2
:1010B000FF031940044B0B4343EA0221014B196023
:1010C00000BF70470CED00E00000FA0570B5044663
:1010D0000D4600266248006800F00700A8420ED2C4
:1010E0005F48006820F0070028435D490860084613
:1010F000006800F00700A84201D0012070BD2078F0
:1011000000F00200022807D15648406820F0F000A5
:10111000A168084353494860207800F00100002886
:101120005DD06068012806D14E48006800F40030A8
:1011300090B90120E2E76068022806D149480068BA
:1011400000F0007040B90120D8E74648006800F080
:10115000020008B90120D1E74248406820F00300AE
:10116000616808433F494860FFF7BEFE0646606875
:10117000012810D108E0FFF7B7FE801B41F288314B
:10118000884201D90320B9E73648406800F00C00D6
:101190000428F0D123E06068022810D108E0FFF7AE
:1011A000A3FE801B41F28831884201D90320A5E7C4
:1011B0002C48406800F00C000828F0D10FE008E04F
:1011C000FFF792FE801B41F28831884201D903204B
:1011D00094E72448406800F00C000028F0D1204833
:1011E000006800F00700A8420ED91D48006820F0F2
:1011F000070028431A4908600846006800F0070005
:10120000A84201D0012079E7207800F004000428EA
:1012100007D11448406820F4E060E16808431149B0
:101220004860207800F00800082808D10D48406880
:1012300020F46050216940EAC1000A49486000F08A
:101240003DF808494968C1F30311074A515CC84099
:10125000064908600020FFF76DFE00204EE7000001
:1012600000200240001002405CA500086001002040
:1012700001480068704700006001002000B5FFF7DA
:10128000F7FF04494968C1F30221034A515CC84091
:1012900000BD0000001002406CA5000800B5FFF77B
:1012A000E7FF04494968C1F3C221034A515CC840C1
:1012B00000BD0000001002406CA50008F0B585B02C
:1012C0000FF26C0C9CE8E01001A8A0E8E0101CA54F
:1012D0002D68009500210022002300240020194DD4
:1012E000696801F00C05F5B1042D02D0082D19D163
:1012F00001E0154819E001ADC1F38346AC5D01F48E
:10130000803555B10F4D6D68C5F340451DF805207A
:101310000D4D6543B5FBF2F302E00C4D04FB05F304
:10132000184602E000BF084800BF00BF05B0F0BD8E
:1013300002030405060708090A0B0C0D0E0F101016
:10134000010200000010024000127A0000093D0076
:10135000F8B504460025207800F00100002878D078
:10136000F848406800F00C0004280CD0F5484068AC
:1013700000F00C00082811D1F248406800F48030D9
:10138000B0F5803F0AD1EF48006800F40030002833
:101390005FD0606800285CD10120F8BD00BF6068A4
:1013A000B0F5803F06D1E748006840F48030E54959
:1013B000086028E0606858B9E248006820F480308E
:1013C000E04908600846006820F4802008601AE0C0
:1013D0006068B0F5A02F0BD1DA48006840F4802097
:1013E000D84908600846006840F4803008600AE088
:1013F000D448006820F48030D2490860084600686C
:1014000020F48020086000BF606888B1FFF76CFDA1
:10141000054606E0FFF768FD401B642801D903205C
:10142000BBE7C848006800F400300028F2D010E0A4
:10143000FFF75AFD054606E0FFF756FD401B6428FE
:1014400001D90320A9E7BF48006800F40030002854
:10145000F2D1207800F00200022857D1B948406844
:1014600000F00C0050B1B748406800F00C000828AC
:1014700018D1B448406800F4803098B9B148006889
:1014800000F0020020B12069012801D0012084E78A
:10149000AC48006820F0F800616940EAC100A94941
:1014A000086033E02069E8B10120A7490860FFF730
:1014B0001BFD054606E0FFF717FD401B022801D97A
:1014C00003206AE79F48006800F002000028F2D07D
:1014D0009C48006820F0F800616940EAC100994921
:1014E000086013E0002098490860FFF7FDFC0546FE
:1014F00006E0FFF7F9FC401B022801D903204CE766
:101500009048006800F002000028F2D1207800F036
:10151000080008282DD1A069B8B101208B490860C6
:10152000FFF7E2FC054606E0FFF7DEFC401B022861
:1015300001D9032031E78348406A00F00200002807
:10154000F2D0012001F0D2FB13E000207F490860B7
:10155000FFF7CAFC054606E0FFF7C6FC401B022861
:1015600001D9032019E77748406A00F002000028FB
:10157000F2D1207800F00400042873D100267148CD
:10158000C06900F0805070B900BF6E48C06940F07B
:1015900080506C49C8610846C06900F080500090D6
:1015A00000BF00BF01266A48006800F48070B0B92F
:1015B0006748006840F4807065490860FFF794FC54
:1015C000054606E0FFF790FC401B642801D9032084
:1015D000E3E65F48006800F480700028F2D000BFA6
:1015E000E068012806D15748006A40F001005549DB
:1015F000086227E0E06858B95248006A20F001000C
:10160000504908620846006A20F00400086219E0A8
:10161000E06805280BD14B48006A40F004004949B6
:1016200008620846006A40F0010008620AE0454886
:10163000006A20F00100434908620846006A20F071
:101640000400086200BFE068A0B1FFF74DFC05464A
:1016500009E0FFF749FC401B41F28831884202D97A
:1016600003209AE622E03748006A00F002000028D2
:10167000EFD012E0FFF738FC054608E0FFF734FC36
:10168000401B41F28831884201D9032085E62D486C
:10169000006A00F002000028F0D1012E05D129488F
:1016A000C06920F080502749C86100BFE069C8B315
:1016B0002448406800F00C00082860D0E069022847
:1016C00048D1002020490866FFF70EFC054606E0D9
:1016D000FFF70AFC401B022801D903205DE61948E8
:1016E000006800F000700028F2D1206AB0F5803F59
:1016F00007D11448406820F40030A168084311491C
:101700004860D4E9080108430E49496821F474117E
:1017100008430C49486001200B490866FFF7E4FBC9
:10172000054607E02DE0FFF7DFFB401B022801D94B
:10173000032032E60348006800F000700028F2D071
:101740001FE00000001002400000424280044242BC
:101750000070004000200C490866FFF7C5FB0546F5
:1017600006E0FFF7C1FB401B022801D9032014E665
:101770000648006800F000700028F2D101E0012066
:101780000BE6002009E60000000042420010024083
:10179000042808D14FF0E021096941F004014FF01D
:1017A000E022116107E04FF0E021096921F0040116
:1017B0004FF0E02211617047704770B5044625462E
:1017C000681EB0F1807F01D301200FE0681E4FF04A
:1017D000E02148610F214FF0FF3001F095F9002022
:1017E0004FF0E021886107200861002070BD10B52E
:1017F000FFF7E2FF10BD10B504460CB9012010BD83
:1018000094F83D0028B9002084F83C00204600F000
:101810000DF8022084F83D00211D206801F0B2FC83
:10182000012084F83D000020E9E7000008B50168C8
:10183000B1F1804F0DD100BF0649C96941F00101E6
:10184000044AD1611146C96901F00101009100BF4C
:1018500000BF08BD0010024001460868C06840F0A3
:1018600001000A68D0600868006840F001000A685A
:1018700010600020704701460868C06820F0010031
:101880000A68D06000BF0868006A41F21112104077
:1018900050B90868006A9210104028B908680068BA
:1018A00020F001000A68106000BF0020704770B58A
:1018B0000446002520684069C0F3C01594F839003B
:1018C00021280ED16DB12068406920F08000216888
:1018D0004861206B10B1206BFEF7A8FF204601F095
:1018E00007FD20684069C0F3801594F83A0022286B
:1018F0000ED16DB12068406920F040002168486138
:10190000606B10B1606BFEF791FF204601F0D0FCD8
:10191000002070BD704701460022002391F8392055
:1019200091F83A3042EA0300704700002DE9F04791
:101930000446206805682068C668206847694FF03B
:101940000008C14605F00F08B8F1000F0AD105F0F4
:10195000200038B106F0200020B1204601F014FD2F
:10196000BDE8F087B8F1000F6DD007F0010018B99D
:1019700006F49070002866D005F0010030B106F43E
:10198000807018B1E06B40F00100E06305F00400E6
:1019900030B107F0010018B1E06B40F00200E063E5
:1019A00005F0020030B107F0010018B1E06B40F023
:1019B0000400E06305F0080030B107F0010018B141
:1019C000E06B40F00800E063E06B68B305F02000D6
:1019D00028B106F0200010B1204601F0D5FC2068A7
:1019E0004069C0F38019E06B00F0080010B9B9F14C
:1019F000000F22D0204601F05BFC2068406900F017
:101A00004000B0B12068406920F040002168486182
:101A1000606B50B11748616B4863606BFEF724FF41
:101A200010B1606B416B88470CE02046FFF772FFF6
:101A300008E02046FFF76EFF04E02046FFF76AFF4C
:101A40000020E0638CE705F0800030B106F08000F4
:101A500018B1204601F0D0FD82E705F0400030B11A
:101A600006F0400018B1204601F032FC78E700BFD4
:101A700076E70000F931000810B504460CB90120E2
:101A800010BDA06900B100E000BF94F8390028B98A
:101A9000002084F83800204600F028F8242084F83C
:101AA00039002068C06820F400502168C8602046D2
:101AB00001F0BEFC2068006920F4904021680861B4
:101AC0002068406920F02A00216848612068C068C9
:101AD00040F400502168C8600020E063202084F8B2
:101AE000390084F83A000020CAE7000010B586B03B
:101AF00004466F492068884277D100BF6D488069ED
:101B000040F004006B4988610846806900F00400D9
:101B1000019000BF00BF00BF0846C06940F400301C
:101B2000C8610846C06900F40030019000BF00BFE2
:101B300004200290022003900320059001200490CD
:101B400002A95D48FFF73CF80820029000200390AE
:101B500002A95948FFF734F82620FFF757FA032265
:101B600011462620FFF75FFA5448554908600020C7
:101B700048600021524881608021C16000210161DC
:101B8000416181614FF40051C161FEF793FF18B1CB
:101B9000AB214CA001F078FE00BF4948606344626D
:101BA00000BF464814304D490860102048600021AD
:101BB0004A4881608021C1600021016141618161E9
:101BC000C161FEF777FF18B1BB213EA001F05CFEBA
:101BD00000BF42482063446200BF03221146262012
:101BE000FFF721FA2620FFF711FA3D4920688842C5
:101BF0005CD100BF2F48806940F008002D49886102
:101C00000846806900F00800019000BF00BF00BFD7
:101C10000846806940F0100088610846806900F03D
:101C20001000019000BF00BF00BF0846C06940F42B
:101C30008020C8610846C06900F48020019000BF80
:101C400000BF081502900220039001200490032099
:101C5000059002A92348FEF7B3FF4FF400600290FD
:101C60000020039002A91F48FEF7AAFF4FF400507E
:101C7000029001200390002004900320059002A907
:101C80001948FEF79DFF19480068C06840F0200021
:101C900016490968C8602720FFF7B8F902221146E3
:101CA0002720FFF7C0F9002001F0E2FD06B010BDCB
:101CB0000044004000100240000801406C00024057
:101CC000400500202E2E5C53595354454D5C5573EE
:101CD0006172745C75736172742E6300FC04002081
:101CE00000480040000C014000100140BC040020EE
:101CF00077B581B00446154694F83A00202850D1B3
:101D0000029800B115B9012004B070BD00BF94F86D
:101D10003800012801D10220F6E7012084F83800BC
:101D200000BF0298A062A5850020E063222084F80D
:101D30003A001D48616B88621C48616BC8621C4890
:101D4000616B08630020616B486302AE32682368F0
:101D5000191D2B46606BFEF7E5FE00BF00200090CA
:101D600020680068009020684068009000BF00BFB5
:101D700000BF002084F8380000BF2068C06840F42D
:101D800080702168C8602068406940F001002168C7
:101D900048612068406940F04000216848610020A7
:101DA000B2E70220B0E700005D320008A33200086D
:101DB0000D32000810B5034693F83A0020282FD1C1
:101DC00001B10AB9012010BD00BF93F83800012805
:101DD00001D10220F7E7012083F8380000BF9962A3
:101DE0009A85DA850020D863222083F83A0000BF64
:101DF000002083F8380000BF1868C06840F4807085
:101E00001C68E0601868406940F001001C6860616F
:101E10001868C06840F020001C68E0600020D2E72D
:101E20000220D0E710B504462749206888420ED129
:101E3000012001F01DFD962002F0A0FF23A001F07B
:101E400025FD962002F09AFF002001F011FD2149A6
:101E50002068884236D12048008800F4004088BBC2
:101E60001D48008800F4804070B11C4800780A28A2
:101E700003D000201849088024E01748008840F467
:101E80000040154908801DE0144800780D2806D14F
:101E90001148008840F480400F49088012E00F4844
:101EA00000780D490988C1F30D010D4A50540A48C4
:101EB0000088401C0849088008460088C72801DDC2
:101EC0000020088010BD000000440040696E746569
:101ED000720000000048004016000020180000209A
:101EE000B403002070472DE9F84304460D4616461A
:101EF0001F464FF0000994F8390020285CD105B145
:101F000016B90120BDE8F88300BF94F83800012815
:101F100001D10220F6E7012084F8380000BF00203C
:101F2000E063212084F83900FEF7DEFF8146A684B5
:101F3000E6842BE0E08C401EE084A068B0F5805F72
:101F400016D14B46002280212046009701F088FBE5
:101F500008B10320D6E7A846B8F80000C0F308008F
:101F600021684860206908B9AD1C0FE06D1C0DE0C8
:101F70004B46002280212046009701F071FB08B1FA
:101F80000320BFE715F8010B21684860E08C0028AA
:101F9000D0D14B46002240212046009701F060FB43
:101FA00008B10320AEE7202084F8390000BF0020EC
:101FB00084F8380000BFA5E70220A3E7704700BF00
:101FC000FEE7000010B500200F4908600F480068C8
:101FD00020F070400D4908600846006840F040500D
:101FE000086000200A49C1F89C01022002F0C6FEE8
:101FF000012005490860022002F0C0FE00200449CB
:10200000C1F8980110BD000098812142000C0140E8
:102010000080214200B585B000BF1E48806940F0B5
:1020200008001C4988610846806900F0080000909B
:1020300000BF00BF00BF0846806940F01000886103
:102040000846806900F01000009000BF00BFC0206B
:1020500001900120029003900320049001A90E48F2
:10206000FEF7AEFD4FF40070019001200290039046
:102070000320049001A90948FEF7A2FD01200849A8
:1020800008600849C1F8980100200749086005B0B8
:1020900000BD000000100240000C01400010014093
:1020A0009C812142008021422401224210B500205F
:1020B0000F4908600F48006820F070400D49086023
:1020C0000846006840F04050086001200A49C1F805
:1020D0009C01022002F052FE012005490860022006
:1020E00002F04CFE00200449C1F8980110BD000028
:1020F00098812142000C01400080214270B50546C4
:1021000000241748006820F0704015490860084610
:10211000006840F000400860002616E000201149E9
:102120000860022002F02AFE01200F49C1F8980140
:102130006006040E0B487C38006808B1601CC4B20D
:10214000012002F01BFE701CC6B2082EE6DB15B99A
:10215000FFF7ACFF01E0FFF735FF204670BD000040
:10216000000C0140988121420080214270B5044654
:102170001548006820F07040134908600846006860
:1021800040F040500860002010490860002517E02A
:10219000E0090E49091D08606006040E022002F0E5
:1021A000EDFD01200A49C1F89801022002F0E6FD88
:1021B000002006490860022002F0E0FD681CC5B25C
:1021C000082DE5DB70BD0000000C01409881214224
:1021D0000080214210B50F48006820F070400D4982
:1021E00008600846006840F04050086001200A4935
:1021F00008600A49C1F89801042002F0BFFD0020E0
:1022000005490860042002F0B9FD00200349C1F827
:10221000980110BD000C01409C81214200802142A8
:1022200010B50F48006820F070400D49086008465E
:10223000006840F04050086000200A4908600A49E0
:10224000C1F89C01042002F099FD012005490860B5
:102250000549C1F89C01042002F090FD10BD00006A
:10226000000C0140988121420080214210B50024D9
:102270001448006820F07040124908600846006861
:1022800040F00040086001200F49086002F076FD30
:1022900001200E49C1F8980102F070FD07E0601CB2
:1022A000C4B2FA2C03DDFFF7BBFF012010BD0648C6
:1022B000803800680028F2D10349091F086000BF78
:1022C000F4E70000000C01409C8121420080214283
:1022D0000146CA1701EB92729210A1EB820292B9E9
:1022E000642091FBF0F200FB121050B94FF4C8705B
:1022F00091FBF0F200FB121008B90120704700209A
:10230000FCE70120FAE70020F8E7000000B585B0FF
:1023100000BF1548806940F01000134988610846E5
:10232000806900F01000009000BF00BF0320019002
:102330000120029003900320049001A90B48FEF7AE
:102340003FFC0220019001200290039003200490A2
:1023500001A90748FEF734FC002201210348FEF7DB
:10236000BDFD05B000BD000000100240001001409E
:10237000000C014010B50446204600F08DF82820DE
:1023800004F0B8FA206028212068FDF7F6FE2068E6
:1023900044622079216808702E49206806F0BCFA52
:1023A0000020C4F89C00C4F8A000C4F8A4000120D8
:1023B000C4F8AC004FF47A70A4F890000121932087
:1023C0000155922001559820045123499420015130
:1023D00004F1900007F06AFA04F1900007F0A8FAFF
:1023E00004F1900007F088FAA0892168088122682A
:1023F000111DA06801F094F9B8B1012001F038FA7C
:10240000962002F0BBFC15A0D4E9021201F03EFABE
:10241000962002F0B3FC002001F02AFAB4F8A820BC
:1024200091B2206806F040FA10E0012001F020FA95
:10243000962002F0A3FC10A0D4E9021201F026FAC3
:10244000962002F09BFC002001F012FA082084F88C
:10245000B00010BD9D7A0008FD8300085443503A37
:1024600020436F6E6E65637420746F206970202541
:10247000733A25640D0A00005443503A20436F6EAE
:102480006E65637420746F20646F6D61696E2025C2
:10249000733A25640D0A000010B504462068B0B1F7
:1024A000012001F0E5F9962002F068FC0AA001F095
:1024B000EDF9962002F062FC002001F0D9F92068C5
:1024C00006F012FA206802F0A9FD0020206004F155
:1024D000900007F02DFA10BD46726565206D656DA0
:1024E0006F72790D0A0000002DE9F0470446884616
:1024F00016461F46DDE9089A012001F0B9F9962039
:1025000002F03CFC3BA001F0C1F9962002F036FC41
:10251000002001F0ADF9242104F15800FDF72DFE53
:102520004046FDF75DFE0546681C04F0E3F9A06532
:10253000691CA06DFDF721FE4146A06DFDF772FEFE
:102540000020A16D48553046FDF74AFE0546681C3F
:1025500004F0D0F9E065691CE06DFDF70EFE314630
:10256000E06DFDF75FFE0021E06D41553846FDF757
:1025700037FE0546681C04F0BDF92066691C206E14
:10258000FDF7FBFD3946206EFDF74CFE0021206E65
:102590004155C4F86C90C4F878A04FF4806004F002
:1025A000A9F920624FF48061206AFDF7E6FD4FF43F
:1025B0008061A162084604F09DF960624FF4806179
:1025C000606AFDF7DAFD4FF48061E16204F15800C2
:1025D000E06100216186A08D82B204F13800616A59
:1025E00005F06CF94FF4006104F1B40000F05AFBFF
:1025F000BDE8F0874D5154545F496E6974436C696E
:10260000656E740D0A0000002DE9F04104460E4687
:1026100017469846012001F02BF9962002F0AEFBF8
:1026200012A001F033F9962002F0A8FB002001F07F
:102630001FF9D0212046FDF7A0FD3046FDF7D0FD63
:102640000546681C04F056F9A060691CA068FDF7F7
:1026500094FD3146A068FDF7E5FD0020A1684855CE
:10266000E76084F80480BDE8F08100004D515454C7
:102670005F496E6974436F6E6E656374696F6E0D4A
:102680000A000000C0F88C107047C1677047C0F89E
:1026900088107047C0F880107047C0F884107047E9
:1026A0002DE9F043ADF2144D04460D4616461F4683
:1026B000DDF83494DDF8308404F14C003B463246BA
:1026C0002946CDE900890290143805F048F9606385
:1026D000606B808898B9012001F0CAF8962002F05A
:1026E0004DFB2DA001F0D2F8962002F047FB002010
:1026F00001F0BEF800200DF2144DBDE8F08301207A
:1027000001F0B6F8962002F039FBD4E93123606B72
:10271000818829A001F0BAF8962002F02FFB002052
:1027200001F0A6F829E0012001F0A2F8962002F0BD
:1027300025FB2FA001F0AAF8962002F01FFB002035
:1027400001F096F84FF4806304AA05A904F1B400DF
:1027500000F09AFA401C80B9012001F089F8962017
:1027600002F00CFB27A001F091F8962002F006FB86
:10277000002001F07DF80020BDE7606B82880168D1
:1027800004F1B40000F0A7FA401C0028CBD020468A
:1027900000F048F80120AEE74D5154543A205175ED
:1027A0006575696E67207075626C69736820666113
:1027B000696C65640D0A00004D5154543A207175DE
:1027C0006575696E67207075626C6973682C206C22
:1027D000656E6774683A2025642C2071756575658F
:1027E0002073697A652825642F2564290D0A000065
:1027F0004D5154543A2051756575652066756C6C61
:102800000D0A00004D5154543A20536572696F759A
:102810007320627566666572206572726F720D0A4A
:102820000000000010B5ADF5826D0446012001F0F6
:102830001FF8962002F0A2FA94F8B01051A001F00F
:1028400025F8962002F09AFA002001F011F814B948
:102850000DF5826D10BD94F8B000062806D007284B
:1028600005D009287ED00F2800D118E086E0204648
:10287000FFF780FD012000F0FBFF962002F07EFABA
:1028800046A0D4E9021201F001F8962002F076FA8F
:10289000002000F0EDFF082084F8B0006EE0012079
:1028A00000F0E6FF962002F069FA43A000F0EEFF88
:1028B000962002F063FA002000F0DAFF04F1B40081
:1028C00000F001FA10B9D4F8A80000B156E04FF4B6
:1028D000806303AA04A904F1B40000F0D5F900282C
:1028E00044D1012000F0C4FF962002F047FABDF861
:1028F0000C20354935A000F0C9FF962002F03EFAC1
:10290000002000F0B5FF04A804F01EFF2065BDF80C
:102910000C1004A804F01CFE4C2108530520C4F838
:10292000A800BDF80C00ADF8040004A80290012036
:1029300000F09EFF962002F021FA4C20025B27A0B7
:10294000216D00F0A3FF962002F018FA002000F09D
:102950008FFFB4F8A8108BB22068DDE9011206F0F1
:102960000BF800E003E00021616307E006E0204689
:10297000FFF792FD204600F043F800BF00BF00BF04
:1029800066E700004D515454205441534B3A207394
:10299000746174653A2025640A0000005443503A7B
:1029A000205265636F6E6E65637420746F3A2025E4
:1029B000733A25640D0A00004D515454205441537C
:1029C0004B20444154410A0044A6000825732C20A2
:1029D000646174614C656E3A25640A004D5154542B
:1029E0003A2053656E64696E672C20747970653A7D
:1029F0002025642C2069643A20253034580D0A00C3
:102A000010B5044604B910BDA06820B1A06802F05A
:102A100005FB0020A060206E20B1206E02F0FEFABF
:102A200000212166A06D20B1A06D02F0F7FA002010
:102A3000A065E06D20B1E06D02F0F0FA0021E165E3
:102A4000206A20B1206A02F0E9FA00212162606A5E
:102A500020B1606A02F0E2FA00216162D4F8B400A9
:102A600030B1D4F8B40002F0D9FA0020C4F8B400B0
:102A7000012000F0FDFE962002F080F908A000F091
:102A800005FF962002F07AF9002000F0F1FED4F85C
:102A90008C0018B12046D4F88C10884700BFB2E7EC
:102AA0006D71747420657869743A0A0008B500BFC6
:102AB0000E48406940F001000C49486108464069F1
:102AC00000F00100009000BF00BF0322114610205B
:102AD000FEF7A9FA1020FEF799FA002211461120FC
:102AE000FEF7A1FA1120FEF791FA08BD001002408E
:102AF00000BFFEE77047000002480068C0F30220F4
:102B0000704700000CED00E010B5002807DA0A0756
:102B1000140E054A00F00F031B1FD45403E00A07EC
:102B2000130E024A135410BD18ED00E000E400E05B
:102B30002DE9F04107460C46164602257E2138460F
:102B400000F011F9401C10B9E81EBDE8F0812FE03B
:102B500020787D2804D07E2803D07F281AD101E078
:102B600000BF00BF7D21384600F0FDF8401C10B9C1
:102B70004FF0FF30E9E714F8012B82F020013846CE
:102B800000F0F1F8401C10B94FF0FF30DDE7A81C51
:102B900085B20CE014F8011B384600F0E4F8401C44
:102BA00010B94FF0FF30D0E7681C85B200BF00BFFE
:102BB000301EA6F101010EB2CAD17F21384600F0C5
:102BC000D2F8401C10B94FF0FF30BEE728B2BCE786
:102BD00010B504462260A3800020E080E1602072EE
:102BE00010BD70B504460D467D2D04D07E2D05D058
:102BF0007F2D10D108E0012020721FE00020E0802E
:102C000020720120607219E0E06808B1E068804736
:102C10000020607270BD607A00B90FE0207A18B1B0
:102C200085F0200500202072E088A188884204DA1F
:102C3000E188481CE0802068455400BF00BFFF20A9
:102C4000E8E7F0B585B006460C4615461F463B46FC
:102C5000224600216846FFF7BBFF0BE09DF81010ED
:102C60006846FFF7BEFF28B9BDF80600288000209F
:102C700005B0F0BD04A9304600F04CF80028EDD0B6
:102C80004FF0FF30F4E770472DE9F04104460D4660
:102C900016461F463B4632462946201DFFF7D1FF08
:102CA000BDE8F08170B504460D46284603F022FECB
:102CB000206029462068FDF760FA2A46201D216819
:102CC00000F041F870BD01460869002801DC0120D0
:102CD00070470020FCE770B504460E4615462AB240
:102CE0003146201DFFF724FF70BD000008B50849DC
:102CF0000968C9084FF47A72B1FBF2F141430091BF
:102D000000BF00BF00994A1E00920029F9D108BDFA
:102D1000600100200246D068002802DC4FF0FF303E
:102D20007047D068401ED0605068431C53600378E1
:102D30000B701369106818445368984201D81068E2
:102D400050600020ECE7034613B109B1022A02DA11
:102D50004FF0FF3070479960596019600020D860CB
:102D60001A6100BFF6E70246D0681369984202DB99
:102D70004FF0FF307047D068401CD0609068431C13
:102D8000936001701369106818449368984201D8E1
:102D9000106890600020EDE770B500260024002543
:102DA0003A4806683604001D006806443848B6FBF9
:102DB000F0F438480088A0423AD036490C8040F2FE
:102DC000B2750EE02846FFF783FA30B1B4F5B77F4D
:102DD00002D3A4F5B77402E006E0A4F26D14681CF7
:102DE00085B2B4F5B67FEDD800BF2B4885800025AD
:102DF00016E029498888FFF76BFA30B1012D04D11C
:102E00001D2C01D31D3C09E00CE02448405DA0428C
:102E100003D82248405D241A00E003E0681C85B214
:102E20001C2CE6D200BF681C1B498871601CC8714D
:102E30001748B6FBF0F100FB11644FF46160B4FB7E
:102E4000F0F0154908704FF46160B4FBF0F100FB3D
:102E500011403C21B0FBF1F00F4948704FF4616024
:102E6000B4FBF0F100FB11403C21B0FBF1F201FB9F
:102E70001200094988700B46DA799979988800F030
:102E80000FF805490872002070BD000018280040A6
:102E90008051010030000020D805002098A40008CF
:102EA000F0B503460C461546642093FBF0F0C6B21D
:102EB000642093FBF0F700FB1730C1B2132E02DD44
:102EC00001F16400C1B20846CF1701EB977701EB1F
:102ED000A707BAB2072092FBF0F700FB172082B2D7
:102EE0005719601EDFF82CC01CF80000384482B26D
:102EF000CF1701EB9777BF10A1EB87071FB9032C02
:102F000001DA501E82B2072092FBF0F700FB172077
:102F1000C0B2F0BD8CA4000810B51148006840682C
:102F200000F0010030B16FF001000D490968486000
:102F3000FFF732FF0A480068406800F0010048B11E
:102F40006FF00200064909684860FFF725FF05A0F9
:102F500000F09CFC6FF0040001490968486010BD56
:102F6000C4050020414C41524D2041210D0A000072
:102F7000704730B58FB0054600240120059000044D
:102F800006900020079002200C90C1030D910E9531
:102F900005A8FEF7DDF904460CB100BFFEE70F20DF
:102FA000009002200190002002904FF48060039076
:102FB0000020049002216846FEF788F804460CB110
:102FC00000BFFEE70FB030BD10B5FDF793FFFEF771
:102FD0000EFC10BD1148006840F001000F49086068
:102FE000084640680E4908400C4948600846006899
:102FF0000C490840094908600846006820F4802010
:1030000008600846406820F4FE0048604FF41F0046
:103010008860C8030449086070470000001002403F
:103020000000FFF8FFFFF6FE08ED00E010B51E48B7
:103030000068C06800F0010080B31C480068406868
:1030400030B11A4A12689068184A12685168884765
:1030500005F0BCFC04461548006840682060134831
:10306000006880686060204601F01CF80F48006826
:10307000807808B907F046F800200B4909684862D3
:1030800000BF0A480068008807490968C862074805
:10309000006801880448C16000BF00BF6FF00100F4
:1030A00001490968086110BDB4120020AC0100207C
:1030B00010B515480068C06800F00100F0B105F0D7
:1030C00085FC0446114800682060002060602046AE
:1030D00000F0E8FF0E48007808B907F061F800201A
:1030E00009490968486200BF4FF47A7006490968C7
:1030F000C86201460448C16000BF00BF6FF0010014
:1031000001490968086110BD8405002028000020DD
:103110002400002010B519480068C06800F00100C4
:1031200028B305F053FC0446154800684068206049
:103130001348006880686060204600F0B3FF1048C4
:103140000068807808B907F073F800200B49096817
:10315000486200BF0A480068008808490968C862D8
:103160000748006801880548C16000BF00BF6FF0D4
:10317000010002490968086110BD0000F412002036
:10318000B001002000220268184B984208D0B0F12C
:10319000804F05D0164B984202D0164B984203D16F
:1031A00022F070024B681A43104B984208D0B0F1DD
:1031B000804F05D00E4B984202D00E4B984203D15F
:1031C00022F44072CB681A4322F080024B691A4302
:1031D00002608B68C3620B688362044B984201D122
:1031E0000B6903630123436170470000002C014019
:1031F000000400400008004070B505466C6A0020DD
:10320000E085E0842046FEF785FB70BD70B506467C
:103210000025746A20684069C0F3C01594F839002D
:10322000212805D125B10020E084204600F060F877
:1032300020684069C0F3801594F83A00222805D12F
:1032400025B10020E085204600F032F8E06B40F028
:103250001000E0632046FEF75DFB70BD70B50546CB
:103260006C6A2868006800F02000B0B90020E08592
:103270002068C06820F480702168C86020684069B8
:1032800020F00100216848612068406920F040007A
:1032900021684861202084F83A002046FEF7C2FDEC
:1032A00070BD70B50446656A2846FEF71BFE70BD0A
:1032B0000168C96821F490710268D16001684969A8
:1032C00021F0010102685161202180F83A10704715
:1032D00010B504462068C06820F040002168C8602E
:1032E000202084F839002046FEF768FE002010BD3B
:1032F0000168C96821F0C0010268D160202180F80E
:1033000039107047F8B504462068006800F01000D6
:1033100010282BD100BF002000902068006800908A
:1033200020684068009000BF00BF2046FEF7BFFA4B
:1033300020680668206846680D4800684668C6F53B
:10334000FA700C4908800CA10D48FCF721FF0546D6
:103350001DB101200B49087001E000F00DFA4FF497
:10336000FA7207492046FEF7C3FC00BFF8BD000013
:103370004005002014000020444F4E45000000008E
:10338000C00100201900002070B5044694F83A00EE
:1033900022284AD1A068B0F5805F13D1A56A2069C0
:1033A00040B920684068C0F308002880A06A801CEB
:1033B000A06219E020684068C0B22880A06A401C62
:1033C000A06211E0206938B920684068C1B2A26AE1
:1033D000501CA062117007E02068406800F07F0177
:1033E000A26A501CA0621170E08D401E80B2E08580
:1033F000C8B92068C06820F020002168C860206833
:10340000C06820F480702168C8602068406920F09E
:10341000010021684861202084F83A002046FEF728
:1034200001FD002070BD0020FCE70220FAE700004B
:103430002DE9F041044600252068006920F4405041
:10344000E1680843216808612169A068084361694F
:10345000084305432068C06841F20C618843284353
:103460002168C8602068406920F44070A169084361
:10347000216848615F49206888425CD1FDF70EFFF2
:1034800000EBC00101EB001061688900B0FBF1F6B0
:10349000FDF704FF00EBC00101EB0010616889003B
:1034A000B0FBF1F06421B0FBF1F000EBC00101EBE7
:1034B0000010A6EB8000322101EB00106421B0FB6C
:1034C000F1F000F0F006FDF7E9FE00EBC00101EBC2
:1034D000001061688900B0FBF1F06421B0FBF1F0ED
:1034E00006EB0016FDF7DAFE00EBC00101EB001061
:1034F00061688900B0FBF1F7FDF7D0FE00EBC00179
:1035000001EB001061688900B0FBF1F06421B0FBB1
:10351000F1F000EBC00101EB0010A7EB80003221BD
:1035200001EB00106421B0FBF1F000F00F0030441B
:10353000216888605BE0FDF7A1FE00EBC00101EBB4
:10354000001061688900B0FBF1F6FDF797FE00EB13
:10355000C00101EB001061688900B0FBF1F064214B
:10356000B0FBF1F000EBC00101EB0010A6EB800016
:10357000322101EB00106421B0FBF1F000F0F00605
:10358000FDF77CFE00EBC00101EB001061688900D3
:10359000B0FBF1F06421B0FBF1F006EB0016FDF793
:1035A0006DFE00EBC00101EB001061688900B0FB0B
:1035B000F1F7FDF763FE00EBC00101EB001061685D
:1035C0008900B0FBF1F06421B0FBF1F000EBC00129
:1035D00001EB0010A7EB8000322101EB0010642109
:1035E000B0FBF1F000F00F00304421688860BDE8C6
:1035F000F081000000380140014691F8390021288F
:103600002CD18868B0F5805F0FD10A6A1088C0F3AA
:1036100008000B685860086918B9086A801C0862BD
:1036200009E0086A401C086205E00B6A581C086241
:1036300018780B685860C88C401E80B2C88458B98E
:103640000868C06820F080000B68D8600868C0680F
:1036500040F040000B68D860002070470220FCE773
:103660002DE9F04104460D4617469846069E21E096
:10367000701CF8B12EB1FDF737FCA0EB0800B0428A
:1036800018D92068C06820F4D0702168C86020680C
:10369000406920F0010021684861202084F8390049
:1036A00084F83A0000BF002084F8380000BF0320EF
:1036B000BDE8F081206800682840A84201D10120BF
:1036C00000E00020B842D3D00020F1E710B5034855
:1036D000FFF718FE0148FEF729F910BD7C04002011
:1036E00010B500240C48FEF721F900BF01E0641C6E
:1036F00000BF0948FEF70FF92028F8D100BF0024C9
:1037000001E0641C00BF012204490348FEF752FB9C
:103710000028F6D100BF10BDBC0400201800002016
:1037200070B504460D46264600211FE0002315E033
:103730003278761C302A08DB392A06DC03EB83005A
:103740004300A2F13000034408E0032901DA2E2AE5
:1037500001D0032900D102E0002070BDE8E700BFDE
:10376000FF2B01DD0020F8E76B54491C0429DDDB49
:103770000120F2E700BFFEE710B5012000F078F865
:10378000962001F0FBFA1D4802881D491DA000F09B
:103790007DF8962001F0F2FA002000F069F805F0BB
:1037A00015F904461F490968086814490A88521C1B
:1037B0001349FCF7C7FC00211A48006800680F4A4B
:1037C000128881540D480088401C16490968888079
:1037D00015482060134800686060204600F062FCD5
:1037E00000200649088000BF03E00021044A11546C
:1037F000401CB0F5FA7FF8DB10BD0000140000207B
:10380000C001002053494D373630303D3D3D3D3EEF
:103810004D43553A25732C206C656E3A25640D0A8C
:10382000000000001C0000206169000870B504461B
:103830000D4642F210732A4621460248FEF753FB1A
:1038400070BD00007C04002010B50446012000F08B
:103850000FF84FF47A7001F091FA204600F016F854
:10386000962001F08BFA002000F002F810BD000055
:10387000014619B90022034B1A6002E00122014BF4
:103880001A607047B401224200BFFEE70FB4054B37
:1038900010B503A9044A029800F030F810BC5DF896
:1038A00014FB000001500008100000200FB4084B6A
:1038B00010B504A902AA039800F020F8044602A952
:1038C000002000F04CFA204610BC5DF814FB00000C
:1038D0005F3D000800487047BC01002002E008C8B6
:1038E000121F08C1002AFAD170477047002001E07A
:1038F00001C1121F002AFBD1704700002DE9FF4FC4
:103900008DB00F460546002606E025280BD0DDE9E0
:103910000F1290476D1C761C28780028F5D111B045
:103920003046BDE8F08F0024A246A1460122EC49B2
:1039300000E0044315F8013F203B02FA03F008427F
:10394000F7D128782A2810D06FF02F022878A0F11C
:103950003001092914D80AEB8A0102EB410144F035
:10396000020400EB010A6D1CF0E701CF5FEA000AD8
:1039700003D544F40054CAF1000A44F002046D1C5B
:1039800028782E2817D115F8010F44F004042A28AE
:103990000ED06FF02F022878A0F1300109290AD843
:1039A00009EB890102EB410100EB01096D1CF2E713
:1039B00057F8049B6D1C28786C280FD006DC4C2827
:1039C00017D068280DD06A2814D104E0742810D0CC
:1039D0007A280FD10DE044F400140AE044F4801476
:1039E00001E044F440146978814202D104F5801466
:1039F0006D1C6D1C2A786E2A1FD00CDC632A31D016
:103A000004DC002A8BD0582A11D1A3E0642A68D0A4
:103A1000692A0CD165E0732A2ED004DC6F2A73D09A
:103A2000702A04D19BE0752A6FD0782A6ED0104698
:103A3000DDE90F129047761C50E1C4F302500228D2
:103A400006D0032809D0042801CF09D0066045E13B
:103A500001CFF117C0E9006140E101CF06803DE1EF
:103A600006703BE117F8040B8DF8000000208DF87C
:103A70000100EB46012003E057F804BB4FF0FF3094
:103A800061074FF0000102D40DE008F10101884602
:103A900049450FDA8045F8DB1BF808100029F4D1FE
:103AA00008E008F1010188468142FADB1BF80810A2
:103AB0000029F6D1DDE90F23AAEB08008146214653
:103AC00000F036F9304400EB080604E0DDE90F129F
:103AD0001BF8010B9047B8F10108F7D22146484680
:103AE000F7E00A21C4F302534FF0000B0891022BB8
:103AF00004D001CFC117032B09D00AE0FF1D27F026
:103B00000707F7E8020108E032E01FE020E000B21A
:103B1000C117042B01D140B2C117031E71F100037C
:103B200007DA4FF0000CD0EB0C006CEB01012D23F9
:103B300002E0230504D52B238DF82430012303E074
:103B4000E30701D02023F7E7984658E00A2110E068
:103B500010210EE010204FF0000B08900CE0102117
:103B60004FF0000B44F004044FF00809089103E003
:103B700008214FF0000B0891C4F30253022B04D02C
:103B800001CF0021032B06D006E0FF1D27F0070719
:103B9000F7E8020103E080B2042B00D1C0B24FF07D
:103BA000000823072BD5702A07D0DDF820C08CF041
:103BB000100C5CEA0B0C05D00EE040238DF824308D
:103BC000012308E050EA010306D030238DF82430A9
:103BD0008DF8252002239846DDF820C08CF0080CD3
:103BE0005CEA0B0C0BD150EA010301D1630706D547
:103BF00030238DF824304FF00108A9F10109582A2B
:103C000004D038A20B9208AA0A920BE03AA2F9E774
:103C10005B46089AFCF744FB0B9B9B5C0A9A521E7E
:103C20000A92137050EA0102F2D10A98ADEB00003B
:103C300000F1200B600702D524F4803401E04FF03E
:103C40000109D94502DDA9EB0B0000E0002000EBE3
:103C50000B0141440890AAEB010AE00306D4DDE918
:103C60000F232146504600F063F806444FF0000948
:103C700008E009A911F80900DDE90F12904709F1E0
:103C80000109761CC145F4DBE0030CD5DDE90F2307
:103C90002146504600F04CF8064404E0DDE90F12DE
:103CA00030209047761C0899481E08900029F5DCC2
:103CB00008E00A980A990078491C0A91DDE90F1278
:103CC0009047761CBBF10001ABF1010BF1DC214602
:103CD0005046DDE90F2300F019F806446D1C1BE681
:103CE00009280100303132333435363738396162D2
:103CF0006364656600000000303132333435363796
:103D00003839414243444546000000002DE9F04166
:103D1000044600251E461746880404D405E03946AB
:103D20002020B0476D1C641EF9D52846BDE8F081FF
:103D30002DE9F041044600251E469046C80301D5F2
:103D4000302700E02027880404D505E041463846A6
:103D5000B0476D1C641EF9D52846BDE8F0810A689D
:103D6000531C0B601070704773B504460D2001F0B2
:103D7000D1FA054601AB2A460D21204600F002F893
:103D80007CBD00002DE9F04F87B0064689461546F8
:103D90001C464FF0000A308804F04EFC834648462B
:103DA00002F0FEF90746012F1CD0C7B9484601F0C2
:103DB000B1FAA84216D00120FFF75AFD962000F074
:103DC000DDFF6BA0FFF762FD962000F0D7FF00201B
:103DD000FFF74EFD4FF0FF3007B0BDE8F08F4FF01A
:103DE000FF30F9E76D4800882844001D0FB9012114
:103DF00000E00021A0EB410069490988884214D9FC
:103E00006748008880302844654908800846008853
:103E100002F070FD82466148028831465046FCF748
:103E200091F9304601F0FAF856460BF101001FFAFD
:103E300080FB5A48008806EB0008584604F0FCFB5B
:103E40003080484604F0F8FB0590BDF81400A8F84F
:103E5000000008F102084FB1284604F0EDFB049081
:103E6000BDF81000A8F8000008F10208B9F10B0F26
:103E700068D2DFE809F06706176721395A672E43D1
:103E80004D00D4E900211046FCF7FEF9CDE9000110
:103E900004F04AFCCDE902012A4602A94046FCF79B
:103EA00051F955E0206804F0E6FB02902A4602A989
:103EB0004046FCF747F94BE0218888B204F0BCFB90
:103EC00000B2ADF808002A4602A94046FCF73AF9CC
:103ED0003EE0208804F0B0FBADF808002A4602A9B5
:103EE0004046FCF72FF933E0206804F0B1FB029064
:103EF0002A4602A94046FCF725F929E0206804F08B
:103F0000A7FB02902A4602A94046FCF71BF91FE0D6
:103F1000D4E90021104604F0BCFBCDE902012A4699
:103F200002A94046FCF70EF912E0D4E90021104640
:103F300004F0AFFBCDE902012A4602A94046FCF796
:103F400001F905E02A4621464046FCF7FBF800BF90
:103F500000BF124800882844001D0FB9012100E06D
:103F60000021A0EB41000D490880002034E700004B
:103F7000506172616D2074797065206469736D6140
:103F800074636820776974682074686520696E704E
:103F90007574206C656E6774680A00009C010020CF
:103FA0009E0100202DE9F74181B004461546002608
:103FB0000027B0461CB9701E04B0BDE8F081D4F8EB
:103FC0000260B4F80080218819480088001D084468
:103FD0002080208802F08EFCC4F802002188D4F8EA
:103FE0000200FCF7CAF8D4F802004246314600F05D
:103FF00089FC07460020009002226946384600F0FE
:1040000081FC0746BDF8080004F016FB029002226E
:1040100002A9384600F076FC074605480288294682
:104020003846FCF78FF8304600F0F8FF0020C3E771
:104030009C01002030B595B004460D46402105A8EE
:10404000FCF79BF814216846FCF797F82146684670
:10405000FCF7E8F8294605A8FCF7E4F805AA694644
:104060000A48FCF784FB401C70B90120FFF700FCF4
:10407000962000F083FE06A0FFF708FC962000F0D3
:104080007DFE0020FFF7F4FB15B030BDDC090020F9
:104090007772697465206669666F206572726F72E7
:1040A000210D0A0070B506460C2002F023FC0446E0
:1040B00014B94FF0FF3070BD00206060A060266032
:1040C0000D48006818B90C4804600020F3E70A485E
:1040D0000068806810B90848056802E00648006872
:1040E000856800E0AD68A8680028FBD1AC60656019
:1040F000A06000BFDFE700002000002010B50246EE
:1041000004E01089401C80B2108101460029F8D0DB
:104110009088801C138A984201DD002010BD0B128C
:104120009488601C9080D06803559488601C9080AF
:10413000D06801550846F1E770B504460E461546AD
:10414000A0882844801C218A884202DD4FF0FF307D
:1041500070BDC5F30721A288501CA080E06881547F
:10416000A288501CA080E0688554A288E168881865
:104170002A463146FBF7E6FFA0882844A080A81C09
:10418000E6E7000010B504463648007890B90120F3
:10419000FFF76EFB962000F0F1FD33A0FFF776FBF2
:1041A000962000F0EBFD0020FFF762FB32A005F047
:1041B000AFFC55E02B480078022803D0294800784E
:1041C00004284DD12E48006888BB2E48FCF7FFFA22
:1041D000002845D12C480078012841D1942002F0D4
:1041E00089FB27490860084602681432016825489F
:1041F000FCF785FA002833D00020234908702048B6
:104200000068143005F084FC0120FFF731FB962094
:1042100000F0B4FD1A48016814311CA0FFF736FB0A
:10422000962000F0ABFD0020FFF722FB18E0FFE72F
:104230000120FFF71DFB962000F0A0FD104801684B
:10424000143112A0FFF722FB962000F097FD00200A
:10425000FFF70EFB10480078401C40B20E49087072
:10426000002010BD500100207374617274207365CA
:104270006E642041540D0A0041540D0A00000000F4
:1042800054010020DC0900205101002073656E6498
:10429000696E673A257300005E0100202DE9FE4338
:1042A00080460E461B4A07CA8DE807004FF0FF37CD
:1042B0000025344600E0641C20787228FBD020786A
:1042C0000A28F8D0002509E05DF825102046FBF704
:1042D0005FFF08B16FB203E0681CC5B2032DF3D3D2
:1042E00000BF27B1012F06D0022F0CD107E001201B
:1042F0000949087008E001200749087004E001201E
:104300000549087000E000BF00BF0348007840B2D4
:10431000BDE8FE83A4A40008510100202DE9FE435E
:1043200080460E461A4A07CA8DE807004FF0FF374D
:104330000025344600E0641C20780D28FBD020784E
:104340000A28F8D0002509E05DF825102046FBF783
:104350001FFF08B16FB203E0681CC5B2032DF3D391
:1043600000BF27B1012F06D0022F09D107E001209D
:104370000849087005E001200649087001E000E0E6
:1043800000BF00BF0348007840B2BDE8FE830000D4
:10439000D8A400085101002010B50A464368036103
:1043A0000276222A01D04E2A13D104E05C2902D1E0
:1043B00043685B1C43604468631C43600368195D89
:1043C00009B12229F2D1046943681B1B5B1E4361BA
:1043D00019E0302A17D100BFD0E90034195D302927
:1043E00001DB392903DD2E2901D0002102E04368D9
:1043F0005B1C43600029EFD103695B1E0361046904
:1044000043681B1B436110BD70B505460C4611483F
:104410000088401E0F490880284601F0C1FEA11CFB
:10442000022202FB00100B494988084409494880D0
:104430000846008860B90848006828B10648006846
:1044400049880844044908600020024908804880DF
:1044500070BD000098010020940100202DE9FE436A
:1044600080460E461A4A07CA8DE807004FF0FF370C
:104470000025344600E0641C20780D28FBD020780D
:104480000A28F8D0002509E05DF825102046FBF742
:104490007FFE08B16FB203E0681CC5B2032DF3D3F1
:1044A00000BF27B1012F06D0022F09D104E001205F
:1044B0000849087005E004E001200649087000E0A2
:1044C00000BF00BF0348007840B2BDE8FE83000093
:1044D00028A50008510100202DE9F04F87B00F46B4
:1044E0001822894901A8FBF72DFE4FF0FF3800265E
:1044F0003C4600E0641C20780D28FBD020780A2878
:10450000F8D000260BE001A850F826102046FBF753
:104510003FFE10B14FFA86F803E0701CC6B2062EBB
:10452000F1D300BFB8F1060F70D2DFE808F0034204
:104530006A6B707175A12046FBF72AFE04461134A0
:104540002046FBF787FE0546B5F57A7F1DDD012085
:10455000FFF78EF9962000F011FC294670A0FFF7B6
:1045600095F9962000F00AFC0020FFF781F97448C5
:10457000006818B100207249096888470120714914
:104580000870801E07B0BDE8F08F6FA12046FBF7D2
:10459000FFFD0446A41C6D496D4A128888182A46FE
:1045A0002146FBF7CFFD6A48008828446849088007
:1045B000A0E0684800F085FC05460DB30120FFF738
:1045C00057F9962000F0DAFB63A0FFF75FF9962019
:1045D00000F0D4FB0020FFF74BF92988686805F04C
:1045E0008DFB29886868FFF721F9686820B1686841
:1045F00000F014FD00206860284600F00FFD002543
:1046000078E077E001204F49087073E071E071E0D5
:104610004FF0000A0FF250190120FFF729F99620F8
:1046200000F0ACFB494953A0FFF730F9962000F0A9
:10463000A5FB0020FFF71CF949464448FBF7A8FDFD
:104640000446DCB90120FFF713F9962000F096FB31
:1046500021464DA0FFF71AF9962000F08FFB0020AD
:10466000FFF706F93648006818B100203449096898
:104670008847012033490870801E83E74846FBF7CE
:10468000AFFD00EB040B5846FBF7E4FD0546C82DD3
:104690001BD00120FFF7ECF8962000F06FFB2946B5
:1046A0003FA0FFF7F3F8962000F068FB0020FFF72B
:1046B000DFF82348006818B10020214909688847BD
:1046C000012020490870801E5CE73AA12046FBF7D4
:1046D0005FFD00F1040A00201D49088001201949EE
:1046E00008701748006818B150461549096888478E
:1046F00000BF00BF00BF384600F090FC0027114803
:10470000007840B23EE7000034A500082B43434840
:10471000524543563A20444154412C312C0000006C
:10472000726573706F6E73652073697A6520697343
:1047300020696C6C6567616C3A2564210A00000091
:1047400048000020510100200D0A0000F40500205F
:104750005A010020DC09002073656E64696E672EC3
:104760002E2E2E2E0A000000485454502F312E3188
:104770000000000068747470207265636569766576
:104780003A25730A00000000496E76616C69642066
:1047900076657273696F6E20696E2025730D0A004D
:1047A000496E76616C6964207374617475733A251F
:1047B000640D0A000D0A0D0A0000000070B50446E1
:1047C0000D4616460120FFF753F8962000F0D6FA62
:1047D0000CA0FFF75BF8962000F0D0FA0020FFF75E
:1047E00047F804EB44000D4901EB8000806838B1C4
:1047F00004EB440001EB8000314682682846904774
:1048000070BD000073656E64207061636B616765E5
:1048100020746F206465766963650A00B00F00201C
:1048200070B504460D46164604EB4400064901EBFC
:104830008000406838B104EB440001EB8000314651
:1048400042682846904770BDB00F002001463029CD
:1048500005DB392903DCA1F13002D0B202E0A1F17D
:104860005702D0B27047000010B5044610220D491F
:1048700004F10900FBF7C9FC88B10120FEF7F8FF3D
:10488000962000F07BFA08A0FFF700F8962000F0D1
:1048900075FA0020FEF7ECFF4FF0FF3010BD00204E
:1048A000FCE7000030110020546F6B656E206572CC
:1048B000726F722E0A0000002DE9FC4104460D467D
:1048C00017464FF000083A212046FBF77FFCB0F175
:1048D000000802D1401EBDE8FC81A8EB0406324668
:1048E00021462846FBF766FC0020A855082208F15F
:1048F00001016846FBF75EFC6846FBF7ABFC3860DD
:104900000020E8E770B504460E4615462A463146B3
:104910002046FBF717FC2C44204670BD2DE9FE43D2
:1049200080460E461C4A07CA8DE807004FF0FF3745
:104930000025344600E0641C20787228FBD02078E3
:104940000A28F8D0002509E05DF825102046FBF77D
:104950001FFC08B16FB203E0681CC5B2032DF3D38E
:1049600000BF27B1012F06D0022F0ED104E0012095
:104970000A4908700AE009E009A12046FBF708FC93
:1049800010B101200549087000E000BF00BF0348D6
:10499000007840B2BDE8FE83B0A4000851010020B9
:1049A000524541445900000010B5044603212046F9
:1049B00000F008F810BD10B5012001F09BFF04467F
:1049C000204610BD2DE9F04107460E460024002583
:1049D000062001F08FFF044600202060A0800C20FC
:1049E0002080208801F086FFC4F802002188D4F8D6
:1049F0000200FBF7C2FBD4F80250012E09D1164881
:104A00008068401C14498860886803F021FEA86013
:104A10000AE0022E08D110480068401C0E490860C8
:104A2000086803F015FEA860032E08D10A48406804
:104A3000401C09494860486803F00AFEA8603846EF
:104A400003F0FAFDE88034202870304603F0F4FDCE
:104A500068802046BDE8F0814011002010B501209B
:104A600001F048FF044600202070204610BD0000E1
:104A700010B5002400200A490880802009490880D8
:104A80000846008801F036FF04460CB9002010BD2E
:104A9000002020800220024908802046F7E700001D
:104AA0009C0100209E0100202DE9FE4380460E4619
:104AB0002B4A07CA8DE807004FF0FF370025344620
:104AC00000E0641C20780D28FBD020780A28F8D05C
:104AD000002509E05DF825102046FBF759FB08B1D9
:104AE0006FB203E0681CC5B2032DF3D300BF27B13A
:104AF000012F10D0022F2BD111E01AA12046FBF775
:104B000047FB0446A01DFBF7A5FB184908700120D0
:104B1000174908701DE001201549087019E00120AF
:104B2000FEF7A6FE962000F029F9214611A0FEF717
:104B3000ADFE962000F022F90020FEF799FEE01D60
:104B4000FBF788FB0949087001200949087000E05B
:104B500000BF00BF0648007840B2BDE8FE830000F9
:104B6000BCA400082B4353513A2000004E00002003
:104B7000510100206373713A25730D0A0000000093
:104B800070B504462646256810A12068FBF700FB97
:104B9000D0B111A12068FBF7FBFA05462D1D284670
:104BA000FBF765FB0E4908800EA12846FBF7F0FADB
:104BB0000546AD1C0C490968086809490A88294658
:104BC000FBF7C0FA012070BD0020FCE752454356B8
:104BD0002046524F4D3A00002B495044000000003F
:104BE0004C0000200D0A0000340000207CB5054672
:104BF0006946284600F0BEFA0646BDF802004FF6A8
:104C0000F871884211D10120FEF732FE962000F0A3
:104C1000B5F81DA0FEF73AFE962000F0AFF8002090
:104C2000FEF726FE04F080FF2CE00120FEF720FEB8
:104C3000962000F0A3F8BDF8021019A0FEF726FE9A
:104C4000962000F09BF80020FEF712FEBDF802103F
:104C5000C8B200F059F904467CB90120FEF708FEFD
:104C6000962000F08BF814A0FEF710FE962000F0BE
:104C700085F80020FEF7FCFD7CBD606810B1304671
:104C80006168884700BFF7E77265636569766520EC
:104C9000612067657420726571756573740A000020
:104CA0000A52656365697665206120636F6D6D6189
:104CB0006E643A25640A00006E6F20737563682085
:104CC000636F6D6D616E642066696E640000000044
:104CD0002DE9FC410446D4F80200218847184FF022
:104CE000000800261BE0BDF80210C8B200F024F94D
:104CF000054685B90120FEF7BBFD962000F03EF881
:104D0000BDF802100AA0FEF7C1FD962000F036F8AB
:104D10000020FEF7ADFD3046A968884700BF694610
:104D2000204600F059FA061EDDD1BDE8FC810000E6
:104D30006F626A656374205B25645D206E6F74200A
:104D4000666F756E6420696E206C6973740A00006A
:104D500010B504460420FCF71BFD0148046010BD9B
:104D60000C00002030B50446002504E04FF47A70B2
:104D700000F004F86D1CA542F8D330BD70B50346B1
:104D800000224FF0E02675690D4E366803FB06F4ED
:104D90004FF0E026B16910E04FF0E026B06988429C
:104DA0000BD0884202D20E1A324402E02E1A0E4470
:104DB00032440146A24200D300E0EDE700BF70BDDF
:104DC0000C00002010B504464CB1D4F8020030B1FC
:104DD000D4F8020000F022F90020C4F802002046B6
:104DE00000F01CF9002410BD10B5044614B1204693
:104DF00000F014F910BD10B5044614B1204600F0BF
:104E00000DF910BD10B504461CB1204600F006F99E
:104E1000002410BD10B5044604B910BD606820B16F
:104E2000606800F0FBF800206060204600F0F6F8B3
:104E3000002400BFF1E7F0B587B004460E461546E2
:104E4000A8B2ADF8140005A9304602F02DFC03907D
:104E5000A8B2ADF816000DF11601304602F0D4FBF1
:104E60000490D4F8880050B1BDF816000090BDF849
:104E70001420DDE903132046D4F88870B84707B042
:104E8000F0BD000010B5044603F0ACFC012809D1C8
:104E9000022006490870064804F04AFD054803F060
:104EA00081FF01E0002010BD00BFFCE78001002071
:104EB000001100206D500008C16801600021818050
:104EC0007047014601F5B460D1F8CC2550F82200B6
:104ED000704700F5B462D0F8C83542F82310704727
:104EE00070B505460748046807E0211D2846FBF712
:104EF0007EF908B9204670BD2468002CF5D1002049
:104F0000F9E70000A80100200246002109E0084856
:104F100010F83100904203D1054800EBC100704702
:104F2000491C044800688142F1DB0020F7E70000DB
:104F30004C110020A0010020024600210CE001EBF2
:104F40004100084B13F82000904204D101EB4100CE
:104F500003EB80007047491C034800688142EEDB88
:104F60000020F7E7CC110020A4010020F0B50C468A
:104F7000059E8588E91E7F292ADD25072D0E02F072
:104F8000010745EAC70503F0030745EA470506F0B0
:104F900001073D43C7683D700D46CF1701EB5767CA
:104FA000FF11A1EBC717FFB247F08007D0F80CC084
:104FB0008CF80170CF1701EB5767C7F3C717D0F80C
:104FC0000CC08CF80270CD1C8580C568056015E0AA
:104FD00025072D0E02F0010745EAC70503F0030778
:104FE00045EA470506F001073D43C7687D70C7687D
:104FF000B9708D1C8580C5686D1C0560F0BD000012
:1050000000BF054A126802F04002002AF9D0C2B27D
:10501000014B1B1D1A6070470048004010B5002866
:1050200021D0114B0022001F196803E0814203D8F0
:105030000A4649680029F9D152B11368841A9C4282
:1050400004D1006818441060104602E0506000E08F
:10505000186039B102680B1A934203D10B681A44E5
:1050600002604968416010BDB401002010B50446DB
:1050700016480078012819D0022821D1A01C38B97F
:10508000012012490870AFF21B0003F099FF0CE0F9
:10509000012C07D103200D490870AFF22F0003F057
:1050A000DBFC02E00A4804F027FC0DE024B9AFF273
:1050B000430003F0D1FC02E0054804F01DFC03E0CE
:1050C000034804F019FC00BF00BF10BD80010020A0
:1050D0000011002010B504460648408820B92088F9
:1050E00003F0AAFA0349088002484188A01C08443A
:1050F00010BD00009801002070B5044600F008F8CB
:105100000546102229462046FBF71CF870BD00001A
:1051100000487047E4050020014890F900007047FE
:105120005001002038B50446002000906946204612
:1051300000F02AF99DF8000038BD70B504460D4610
:10514000208803F079FA2880608803F075FA688077
:10515000A08803F071FAA880201D70BD1CB504461C
:105160000021009101916946204600F00DF9DDE92A
:1051700000011CBD2DE9F04105460C4655F8020F13
:1051800000F10C062F68B86803F062FA0B498860DA
:10519000308803F051FA2080708803F04DFA608067
:1051A000B08803F049FAA080F08803F045FAE08067
:1051B00055F802091230BDE8F081000040110020CE
:1051C00070B5044614B94FF6FF7070BDD4F80250A4
:1051D000688803F031FAF8E72DE9F04104460D46FE
:1051E00000260027164800682188884204D0144809
:1051F00000682188884204DD002011490860BDE86C
:10520000F0810F48006858B90D4800680C300C490F
:105210000860D4F80270B86803F01AFA09494860C7
:10522000D4F8020006490968461805480068801D40
:105230000349086029463046FFF77FFFDFE700009B
:1052400094010020401100202DE9F04707460D464B
:1052500014461E464FF0000938882880288803F03D
:10526000EBF92880288800F09BFF8046B8F1010FF9
:105270000BD178882080208803F0DEF920802288F6
:10528000391D3046FAF75EFF36E0288800F042F814
:10529000208007F10209228849463046FAF752FF7A
:1052A00028880E2826D2DFE800F02507141D2019D3
:1052B0000E1E21180D25251FD6E90021104603F0EA
:1052C00033FA18E000BFD6E90021104603F0E1F9F7
:1052D00011E0306803F0CFF90DE000BF306803F053
:1052E000B7F908E000BF00BF05E000BF308803F059
:1052F000A3F900E000BF00BF20883844001DB8F1CA
:10530000000F01D1012100E00021A0EB4100BDE828
:10531000F087000010B504460E2C1AD2DFE804F026
:1053200019070B0F130D0910140C0816171100BFE5
:1053300000BF082010BD00BF00BF0420FAE700BF77
:1053400000BF0120F6E700BF0220F3E700BF002006
:10535000F0E70120FEF78CFA9620FFF70FFD05A07D
:10536000FEF794FA9620FFF709FD0020FEF780FA79
:10537000FF20DFE7556E6B6E6F77206461746120EC
:10538000747970652E0A00007CB505460C46002035
:10539000019000902846FFF79DFE064623466A4688
:1053A00001A93046FFF750FFBDF80010BDF804001A
:1053B000FFF72AF87CBD00002DE9FF4180460E462C
:1053C000264B0FCB8DE80F004FF0FF3700253446FA
:1053D00000E0641C20780D28FBD020780A28F8D043
:1053E000002509E05DF825102046FAF7D1FE08B146
:1053F0006FB203E0681CC5B2042DF3D300BF37B110
:10540000012F0BD0022F0AD0032F1FD10EE0012055
:105410001349087003201349087018E017E00120B1
:105420000F49087003200F49087010E00120FEF7B3
:105430001FFA9620FFF7A2FC0BA0FEF727FA962092
:10544000FFF79CFC0020FEF713FA00E000BF00BF4E
:105450000348007840B204B0BDE8F081C8A4000859
:1054600051010020500100204E65740D0A0000001B
:105470002DE9FC4180460E46294903C9CDE90001CA
:105480004FF0FF370025344600E0641C20780D28DB
:10549000FBD020780A28F8D022480078D0B90F2213
:1054A00021462148FAF74EFE00201F49C87301200B
:1054B000FEF7DEF99620FFF761FC1B491BA0FEF703
:1054C000E5F99620FFF75AFC0020FEF7D1F90120FC
:1054D00014490870002509E05DF825102046FAF708
:1054E00057FE08B16FB203E0681CC5B2022DF3D3BA
:1054F00000BF17B1012F08D103E001200F49087048
:1055000007E001200D49087003E001200B490870F5
:1055100000BF00BF0948007840B2BDE8FC81000030
:10552000E4A4000858010020E4050020675F6965D5
:105530006D695F6275663A257300000051010020B5
:105540002DE9F04105460E460024002734460DE0C3
:105550006078FFF77BF980462078FFF777F948EA13
:105560000010C2B238467F1C2A54A41C20780028A0
:10557000EED1BDE8F08100002DE9F043A9B0064668
:105580007048006830B16F480068FFF747FD0020A1
:105590006C4908603EB96FF002006B4909688847A2
:1055A00029B0BDE8F0830120FEF762F99620FFF7ED
:1055B000E5FB314665A0FEF769F99620FFF7DEFBB3
:1055C0000020FEF755F93046FAF70AFE401C84B277
:1055D000204601F08FF9054621462846FAF7CDFD11
:1055E000224631462846FAF7ADFD2846FAF7F8FD7F
:1055F00081464A46294620A800F003FF00208DF886
:10560000500056E0B8F14E0F53D155A120A800F03C
:1056100000FF50B920A800F05AFE20A800F057FE65
:1056200020A800F03AFE074643E04FA120A800F072
:10563000F0FE58B920A800F04AFE20A800F047FE6E
:10564000202218A920A800F001FE32E048A120A8DD
:1056500000F0DFFE68BB23E0B8F14E0F20D146A179
:1056600020A800F0D6FE58B920A800F030FE20A8EF
:1056700000F02DFE202210A920A800F0E7FD0FE089
:1056800041A120A800F0C5FE50B920A800F01FFEDF
:1056900020A800F01CFE4022694620A800F0D6FD9C
:1056A00020A800F014FEB0F1000802D023980128D1
:1056B000D2DC20A800F00BFEB0F10008A2D115B199
:1056C0002846FFF7ABFCC7B10120FEF7D1F89620C2
:1056D000FFF754FB18A92FA0FEF7D8F89620FFF784
:1056E0004DFB0020FEF7C4F81748006820B16FF0AA
:1056F000020015490968884752E710A92C48FFF7AE
:105700001FFF0120FEF7B4F89620FFF737FB69462C
:1057100028A0FEF7BBF89620FFF730FB0020FEF72D
:10572000A7F869462DA003F0CFFA10A930A003F026
:10573000CBFA0548006818B1012003490968884779
:1057400000BF2DE7740100207001002072657370A6
:105750006F6E73653D25730A28656E64290A000023
:10576000636F6465000000006D65737361676500B9
:1057700064617461000000006163636573735F744A
:105780006F6B656E000000006163636573735F613A
:1057900064647200646576696365206C6F67696E26
:1057A000206661696C65643A2025730A0000000078
:1057B00068010020646576696365206C6F67696EB7
:1057C00020737563636573732C2061636365737302
:1057D0005F61646472203A2025730A0070616E6410
:1057E0006F5F6163636573735F616464720000007F
:1057F00070616E646F5F6163636573735F746F6B19
:10580000656E00002DE9F047C8B005469348006872
:1058100030B192480068FFF701FC00208F49086012
:10582000CDB90120FEF724F89620FFF7A7FA8CA047
:10583000FEF72CF89620FFF7A1FA0020FEF718F8E3
:105840008D48006838B14FF0FF308B4909688847B0
:1058500048B0BDE8F0870120FEF70AF89620FFF770
:105860008DFA294685A0FEF711F89620FFF786FAF3
:105870000020FDF7FDFF2846FAF7B2FC401C84B279
:10588000204601F037F8064621463046FAF775FC07
:10589000224629463046FAF755FC2846FAF7A0FC7E
:1058A0008246524629463FA800F0ABFD67E0B8F1BA
:1058B0004E0F64D176A13FA800F0ABFD50B93FA8D0
:1058C00000F005FD3FA800F002FD3FA800F0E5FC58
:1058D000C7B254E070A13FA800F09BFD58B93FA8A3
:1058E00000F0F5FC3FA800F0F2FC202237A93FA809
:1058F00000F0ACFC43E06AA13FA800F08AFD00285C
:105900003DD133E0B8F14E0F30D167A13FA800F090
:1059100080FD50B93FA800F0DAFC3FA800F0D7FCAA
:105920003FA800F0C7FC814620E062A13FA800F03C
:1059300070FD58B93FA800F0CAFC3FA800F0C7FCB2
:1059400060221FA93FA800F081FC0FE05DA13FA8E5
:1059500000F05FFD50B93FA800F0B9FC3FA800F08F
:10596000B6FC602207A93FA800F070FC3FA800F039
:10597000AEFCB0F1000802D042980128C2DC3FA87A
:1059800000F0A5FCB0F1000891D116B13046FFF748
:1059900045FBC7B10120FDF76BFF9620FFF7EEF93D
:1059A00037A94BA0FDF772FF9620FFF7E7F900201B
:1059B000FDF75EFF3048006828B14FF0FF302E49F8
:1059C0000968884744E70120FDF752FF9620FFF75A
:1059D000D5F907AB1FAA494644A0FDF757FF96200B
:1059E000FFF7CCF90020FDF743FF4A464DA101A87F
:1059F000FDF75CFF0120FDF73BFF9620FFF7BEF9A6
:105A000049A0FDF743FF9620FFF7B8F90020FDF706
:105A10002FFF01A94DA003F057F91FA94FA003F0D4
:105A200053F907A952A003F04FF90120FDF720FF19
:105A30009620FFF7A3F953A0FDF728FF9620FFF764
:105A40009DF90020FDF714FF0B48006818B10020F5
:105A500009490968884700BFFAE600007C01002078
:105A600068747470207265717565737420666169FD
:105A70006C65640A00000000780100207265737094
:105A80006F6E73653D25730A28656E64290A0000F0
:105A9000636F6465000000006D6573736167650086
:105AA00064617461000000006465766963655F6924
:105AB000640000006465766963655F7365637265A1
:105AC000740000006465766963655F6B657900004A
:105AD00064657669636520726567697374657220B1
:105AE0006661696C65643A2025730A0064657669AD
:105AF000636520726567697374657220737563638B
:105B00006573732C2069643A2025642C20736563C7
:105B1000726574203A2025732C206B6579203A2019
:105B200025730A0025640000736176696E6720643E
:105B3000657669636520696E666F20746F20737483
:105B40006F726167652E2E2E0A00000070616E6410
:105B50006F5F6465766963655F69640070616E6438
:105B60006F5F6465766963655F7365637265740012
:105B700070616E646F5F6465766963655F6B65799C
:105B800000000000646F6E652E2E2E0A00000000DB
:105B90002DE9FF5F0F46944BD3E90020D3E90213B0
:105BA00001AC0BC400924FF0FF3900263C4600E0E8
:105BB000641C20780D28FBD020780A28F8D0002615
:105BC0000AE05DF826102046FAF7E2FA10B14FFA23
:105BD00086F903E0701CC6B2042EF2D300BFB9F1FF
:105BE000000F09D0B9F1010F2BD0B9F1020F6AD023
:105BF000B9F1030F7ED16AE07C48FFF762F90546F0
:105C0000F5B10120FDF734FE9620FFF7B7F878A034
:105C10006968FDF73BFE9620FFF7B0F80020FDF71E
:105C200027FE29886868FDF701FE686820B168686A
:105C3000FFF7F4F9002068602846FFF7EFF9002528
:105C4000CDE070A12046FAF7A3FA044610342046AE
:105C5000FAF700FB05460120FDF70AFE9620FFF744
:105C60008DF829466CA0FDF711FE9620FFF786F807
:105C70000020FDF7FDFD42F2107085420FDD6C48FB
:105C8000006818B100206A490968884700206949FE
:105C900008700846007840B204B0BDE8F09F66A1E5
:105CA0002046FAF775FA0446A41C6449644A12882F
:105CB00088182A462146FAF745FA614800882844A0
:105CC0005F4908808BE001205A49087087E04FF057
:105CD00000080FF2701A0120FDF7CAFD9620FFF7A9
:105CE0004DF856495AA0FDF7D1FD9620FFF746F82A
:105CF000002000E072E0FDF7BBFD51464F48FAF787
:105D000047FA0446ECB90120FDF7B2FD9620FFF7F3
:105D100035F8214652A0FDF7B9FD9620FFF72EF881
:105D20000020FDF7A5FD4248006818B10020404959
:105D30000968884700203F4908700846007840B24B
:105D4000AAE75046FAF74CFA00EB040B5846FAF76C
:105D500081FA0546C82D1DD00120FDF789FD96204A
:105D6000FFF70CF8294644A0FDF790FD9620FFF7B9
:105D700005F80020FDF77CFD2D48006818B10020D3
:105D80002B490968884700202A490870084600788E
:105D900040B281E741A12046FAF7FAF900F1040880
:105DA0000120FDF765FD9620FEF7E8FF41463DA086
:105DB000FDF76CFD9620FEF7E1FF0020FDF758FD92
:105DC00000201F49088001201A49087018480068FF
:105DD00018B1404616490968884700E000BF00BF77
:105DE0001448007840B257E74CA50008DC090020B1
:105DF00073656E64696E6720446174613A25730D42
:105E00000A0000002B43485454504143543A204464
:105E10004154412C00000000726573706F6E736511
:105E20002073697A65206973203A2564210A00008D
:105E300048000020510100200D0A0000F405002058
:105E40005C010020485454502F312E3120000000B6
:105E500068747470207265636976653A25730A0008
:105E6000496E76616C69642076657273696F6E2025
:105E7000696E2025730A0000726573706F6E73651A
:105E800020636F6465206572726F722069732025CC
:105E9000642C206E6F742032303000000D0A0D0A21
:105EA0000000000067657420687474702072657368
:105EB000706F6E73653A2573000000002DE9F041A4
:105EC00004460D4616461F460D48006A401C0C4904
:105ED0000862086A02F0BCFBA060342020704620F3
:105EE0006070287802F0A8FBE080384602F0A4FB3E
:105EF000A080304602F0A0FB60800020BDE8F08169
:105F00000C11002010B596B0342109A8FAF735F924
:105F10001AA002F0CDFE0446FAF7A9F9C117CDE99F
:105F200009011A4903C9CDE912010120FDF7A0FCBE
:105F30009620FEF723FF16A0FDF7A8FC9620FEF79B
:105F40001DFF0020FDF794FC082112A803F084FE39
:105F500024220DA96846FAF7F5F809A80FC803F03E
:105F6000C7FA41F288300C490880012088700B483C
:105F700048600220C87016B010BD000070616E64E9
:105F80006F5F6465766963655F696400680100201E
:105F9000746F6B656E3A0A00F4100020619A000875
:105FA00001460320888070472DE9F04104460D46E4
:105FB000E88802F041FB207003F0DEFC064602F0A8
:105FC00068FBC4F80100C4F805101022034904F16D
:105FD0000900FAF7B7F80020BDE8F0813011002081
:105FE00010B503A105A0FEF725F80648007810BDFE
:105FF00041542B4353510D0A0000000041542B43E0
:10600000535100004E0000202DE9F04385B0814639
:106010000F4614224F496846FAF794F84FF0FF38BC
:1060200000263D4600E06D1C28780D28FBD028781E
:106030000A28F8D000260AE05DF826102846FAF76C
:10604000A7F810B14FFA86F803E0701CC6B2052E0F
:10605000F2D300BFB8F1050F73D2DFE808F00326D2
:10606000335864003C48006860B13B4800680068F1
:1060700040B1394909680868FEF7D0FF0020364969
:106080000968086034480068FEF7C8FF00203249FC
:1060900008600120314908703148006820B10021B2
:1060A00008462F4A126890474CE02D48006828B1F6
:1060B0004FF0FF3100202A4A1268904701202749FB
:1060C00008703FE02748FEF7FCFE04460120FDF77C
:1060D000CFFB9620FEF752FE214623A0FDF7D6FB0C
:1060E0009620FEF74BFE0020FDF7C2FB74B121881D
:1060F0006068FDF79BFB606820B16068FEF78EFF6B
:10610000002060602046FEF789FF00241AE001208D
:10611000124908701248006820B100210846104A50
:10612000126890470EE00E48006828B14FF0FF312A
:1061300000200B4A1268904701200849087001E0CE
:10614000FFE700BF00BF0548007840B205B0BDE8DA
:10615000F083000014A50008340000205101002045
:106160003C000020DC09002073656E64696E672EB8
:106170002E2E2E2E2C25702C0A00000008B5074864
:106180000068401C30B9012000909DF800000349D0
:10619000086000BF0148006808BD000090010020B1
:1061A00010B504460E2C17D2DFE804F016070809D4
:1061B0000A0B0C0D0E0F1013141100BF00BF00BF0F
:1061C00000BF00BF00BF00BF00BF00BF00BF002076
:1061D00010BD00BF0120FBE70120FDF749FB962021
:1061E000FEF7CCFD05A0FDF751FB9620FEF7C6FD9E
:1061F0000020FDF73DFBFF20EAE70000556E6B6EC7
:106200006F77206461746120747970652E0A0000D4
:1062100010B501460A48006880B10A4800680A4A79
:10622000126890420ADA074803680068401C054C6F
:10623000206003480068C154084610BD0020FCE7F8
:10624000840100208C0100208801002030B5034625
:106250000C46187E08B9002030BD5869904201DB19
:10626000501E00E058690246002105E01D690D44FA
:106270001868405D6054491C9142F7DB002060546F
:10628000187EE9E70146C86808B900207047C86869
:10629000401E01F11A02105CF8E710B50446207E9A
:1062A000302801D0002010BD226921688818F9F734
:1062B000D1FFF8E710B50446207E302801D0002039
:1062C00010BD226921688818F9F7D1FFF8E770B589
:1062D0000546284603F064FDD5E90001465C2846E2
:1062E000FFF7D0FFC4B26868401C68605B2E64D0C2
:1062F00006DC222E4AD02C2E38D03A2E6FD12FE039
:106300005D2E21D07B2E02D07D2E68D105E0314656
:10631000284603F061FB304670BD3A2C08D1287E38
:1063200030B1284603F02BFB2846FFF7ABFFC4B281
:106330007B2C03D1284603F022FB03E00120687682
:106340000020E9E73046E7E75B2C03D1284603F05D
:1063500016FB03E0032068760020DDE73046DBE72C
:106360003146284603F038FB3046D5E73A2C05D1B4
:10637000287E18B1284603F002FB05E05B2C03D011
:10638000012068760020C7E73046C5E77B2C03D0A4
:106390005B2C01D03A2C0AD17B2C01D14E2000E09D
:1063A0003046064601462846FDF7F6FF03E0052085
:1063B00068760020B0E73046AEE77B2C03D05B2C3C
:1063C00001D03A2C04D13146284603F005FB03E006
:1063D0000220687600209FE730469DE7FFE73A2CD1
:1063E00001D05B2C09D1392E07DC302E05DB3021A2
:1063F0002846FDF7D1FF30208EE700BF00BF002008
:106400008AE70160826000234360C360437683763D
:10641000704770B504460D46207E10B94FF0FF302E
:1064200070BD23692068C11828466269F9F703FF27
:10643000F6E700002DE9F041044694F8400054F8D6
:1064400020502878492857D004DC22284FD04328F0
:106450007ED156E05B2802D07B2879D100BF2F4641
:1064600094F8401004F1280030F811602EB9287813
:10647000E16B88470A20E16B88477878B04207DCF7
:106480000A20E16B88472A78901CE16B884761E01D
:10649000002E05DD2C20E16B88470A20E16B884740
:1064A00028787B280ED1786850F83610204600F006
:1064B0009BF83A20E16B8847786800EBC600D0F87B
:1064C000048002E0786850F8268014F8400F401CE1
:1064D0002070002114F8402904F1280020F812103F
:1064E00094F8400044F820800120BDE8F081204667
:1064F000696800F079F82DE02046696800F04DF8F1
:1065000028E02F4694F8401004F1280030F81100DC
:1065100008B900206064786820B91CA1204600F00A
:1065200063F814E020467968884780B194F84010F9
:1065300004F1280030F81100401C81B294F840208A
:1065400004F1280020F812100120CEE700E001E05D
:106550000020CAE700BF94F84000002813DD14F8BB
:10656000400F401E207014F8401904F1280030F844
:106570001100401C81B294F8402004F1280020F85A
:1065800012100120B1E70020AFE70000000000007A
:10659000002180F8401001857047FEB506460C4684
:1065A000002C03DA2D20F16B88476442092500BFD7
:1065B0000A2094FBF0F100FB11403030C2B22846B3
:1065C0006D1E0DF800200A2094FBF0F4002C01DD74
:1065D000002DEDDA03E01DF80500F16B8847681C1B
:1065E00005460A28F7D3FEBD70B505460C462220A5
:1065F000E96B88476CB109E02078222802D15C2041
:10660000E96B884714F8010BE96B8847207800286C
:10661000F2D12220E96B884770BD002101707047DC
:1066200010B5FBF773FE10BD0EB5FFF7F9FF044A76
:1066300007CA8DE807009DE8070003F0F7F90EBDD3
:10664000A0A6000870B505467DB90120FDF710F938
:106650009620FEF793FB15A0FDF718F99620FEF79C
:106660008DFB0020FDF704F970BDFEF7A4F9044688
:106670002046FFF7D2FF21782846FDF775FB78B159
:106680000120FDF7F5F89620FEF778FB0FA0FDF747
:10669000FDF89620FEF772FB0020FDF7E9F8E3E72E
:1066A0002046FEF7A1FB00BFDEE7000063726561D4
:1066B000746520666972737420746C7620706172E0
:1066C000616D206661696C65640D0A006164642017
:1066D0006E65787420746C76206661696C65640DF3
:1066E0000A00000070B50546FEF765F90446284625
:1066F000FEF718FD2070204600F004F82046FEF753
:1067000073FB70BD0178014A11607047800122421D
:1067100038B50120FDF7ACF89620FEF72FFB25A039
:10672000FDF7B4F89620FEF729FB0020FDF7A0F84E
:10673000012269460B20F9F742FF0120FDF798F886
:106740009620FEF71BFB9DF8001023A0FDF79EF896
:106750009620FEF713FB0020FDF78AF8002414E0D2
:10676000842000F0C7F8054604EB44110C2202EB2C
:10677000810188B284222946F9F721FF2148006867
:10678000286020480560601CC4B29DF80000844267
:10679000E6DB0120FDF76CF89620FEF7EFFA1AA071
:1067A000FDF774F89620FEF7E9FA0020FDF760F88F
:1067B00038BD00006C6F6164696E6720636F6E6640
:1067C000696720646174612066726F6D20666C6118
:1067D00073682E2E2E0A000072656164696E672050
:1067E000636F6E6669672066726F6D20666C617399
:1067F000682C206B657920636F756E743A25642E62
:106800002E2E0A00A8010020646F6E652E2E2E0A1F
:106810000000000088B0FAF779FB4FF4E010FCF7B5
:10682000A8FB4820FEF794FA4FF4E13003F008FD8E
:106830004FF4E13003F03EFDF9F7BDFE08E03220F1
:10684000FEF790FA0120264908603220FEF78AFA06
:10685000F9F79AFE0028F2D11F226946F9F7AFFE38
:1068600001201F490860FFF7DFFE37E0FEF754FC08
:10687000B0F1FF3F02D100F0E9FB21E0FEF74CFC54
:10688000012802D100F05CFB1AE0FEF745FC03286A
:1068900016D1042003F0DAF90120FCF7E9FF962075
:1068A000FEF76CFA0FA0FCF7F1FF9620FEF766FAF0
:1068B0000020FCF7DDFF00200949086002F098FC89
:1068C00008E0206810B1D4E90010884714B12046D0
:1068D000FEF7A0FA03F060F8041EF2D1C6E700004C
:1068E00080012242496E6974204765747761790D91
:1068F0000A000000F0B50B30154D20F00701002410
:10690000144A0FE003688B420BD38B4205D95E1A01
:1069100043184768C3E9006700E04368136002C09A
:1069200004E0021D10680028ECD12046002802D1A6
:10693000286808B10020F0BD064A07481060074AE1
:10694000121A22F00702C0E9002401202860D7E7CC
:10695000B8010020B40100203C130020383300208F
:10696000F8B50646002000903446A08803281DDABA
:106970000120FCF77DFF9620FEF700FA43A0FCF70C
:1069800085FF9620FEF7FAF90020FCF771FF54B15D
:10699000206820B12068FEF741FB002020602046DF
:1069A000FEF73CFB00244FF0FF30F8BD4148007873
:1069B000B0B941A12068F9F7EBFB88B10120FCF7E1
:1069C00057FF9620FEF7DAF93CA0FCF75FFF962010
:1069D000FEF7D4F90020FCF74BFF01203549087081
:1069E00034480078022803D03248007804283ED189
:1069F00000253A48006810B300BF1DE0384850F841
:106A0000351036480068F9F7F2FBA0B9344800EBBE
:106A1000C5002168426868469047324908700846B8
:106A20000078012806D12D480068FEF7F7FA00200B
:106A30002A49086002E06D1C182DDFD316E02046BD
:106A4000FEF79EF801280ED12748006870B127484C
:106A50000068042201680020234B1B68984700202F
:106A60002349088002E0204603F060FC00BF54B1D7
:106A7000206820B12068FEF7D1FA0020206020466F
:106A8000FEF7CCFA002400208FE700006D6F6475DC
:106A90006C6520726573706F6E7365206E6F742005
:106AA000656E6F756768206C656E677468210D0A86
:106AB00000000000500100204F4B0000746865206A
:106AC0002261742220636D6420726573706F6E732F
:106AD0006520224F4B220D0A0000000054010020C7
:106AE0005000002051010020400000203400002010
:106AF0004C0000202DE9F74FDAB004468A4692494F
:106B00005C98086040214AA8F9F737FB40213AA871
:106B1000F9F733FB4FF0500807228CA12046F9F714
:106B20008AFB08B9012000E000203990082289A1E1
:106B30002046F9F780FB08B9012000E000203890DA
:106B4000399808B1E41D17E0389818B1083440F2BC
:106B5000BB1811E00120FCF78BFE9620FEF70EF922
:106B60007FA0FCF793FE9620FEF708F90020FCF7C3
:106B70007FFE5DB0BDE8F08F2F212046F9F726FBA0
:106B8000054625B900212046F9F720FB05463A21A4
:106B90002046F9F71BFB0646AE4200D900262EB967
:106BA0002A1B21464AA8F9F7CDFA10E0701CF9F724
:106BB00051FB8046B8F1000F00D1DAE7321B2146C5
:106BC0004AA8F9F7BFFA0020311B4AAA5054002006
:106BD000291B4AAA50542046F9F702FB83464AA8CB
:106BE000F9F7FEFAABEB00000246294602903AA8FC
:106BF000F9F7A8FA0120FCF73BFE9620FEF7BEF855
:106C00004AA95FA0FCF742FE9620FEF7B7F80020E5
:106C1000FCF72EFE0120FCF72BFE9620FEF7AEF8C7
:106C20003AA95BA0FCF732FE9620FEF7A7F80020F9
:106C3000FCF71EFE0120FCF71BFE9620FEF79EF8D7
:106C4000414657A0FCF722FE9620FEF797F8002059
:106C5000FCF70EFE56A15AA0FDF7ECF95BA15FA070
:106C6000FDF7E8F9402128A8F9F787FA4AAB012295
:106C70005DA128A8CDF80080FCF718FE0120FCF7E4
:106C8000F7FD9620FEF77AF828A95EA0FCF7FEFD36
:106C90009620FEF773F80020FCF7EAFD28A95FA014
:106CA000FDF7C8F9802108A8F9F767FA142103A8AD
:106CB000F9F763FA5046F9F793FA83465A465AA110
:106CC00008A8FCF7F3FD0820FFF714FE07464FF471
:106CD0000070FFF70FFE786008A8CDE9010ACDF833
:106CE00000804AAB3AAA5D497868FCF7DFFD81462F
:106CF000A7F800900120FCF7BBFD9620FEF73EF8B8
:106D00004A4657A07968FCF7C1FD9620FEF736F891
:106D10000020FCF7ADFD4B46012257A103A8FCF76C
:106D2000C5FD03A959A0FDF785F939465A48FEF774
:106D3000D0F85AA15DA0FDF77DF95FA162A0FDF733
:106D400079F900BF15E700004800002068747470EE
:106D50003A2F2F0068747470733A2F2F00000000D0
:106D600075726C206973206E6F7420687474703A49
:106D70002F2F206F722068747470733A2F2F0000C9
:106D8000686F73745F6E616D653A25730A00000069
:106D9000687474705F706174683A25730A0000004B
:106DA000687474705F706F72743A25640A00000032
:106DB00041542B4343485345543D310D0A000000D4
:106DC00041542B43434853455400000041542B4346
:106DD000434853544152540D0A00000041542B4380
:106DE000434853544152540041542B4343484F505D
:106DF000454E3D25642C222573222C25642C310D13
:106E00000A000000726561647920746F20687474F0
:106E10007020706F73743A257300000041542B4347
:106E200043484F50454E0000436F6E74656E742D9D
:106E3000547970653A6170706C69636174696F6EE2
:106E40002F6A736F6E0D0A436F6E74656E742D4CEE
:106E5000656E6774683A2025640D0A0074A90008FD
:106E60006874747020706F73743A25732C206C658D
:106E70006E3A25640000000041542B4343485345BB
:106E80004E443D25642C25640D0A000041542B43DB
:106E9000434853454E440000DC09002041542B4335
:106EA0004348434C4F53453D310D0A0041542B4359
:106EB0004348434C4F53450041542B43434853549C
:106EC0004F500D0A0000000041542B4343485354D7
:106ED0004F500000F0B58DB007460E46144608200E
:106EE000FFF708FD05462C802046FFF703FD68608C
:106EF000224631466868F9F725F92346012207A1A1
:106F000001A8FCF7D3FC01A909A0FDF793F82946D5
:106F10000A48FDF7DEFF0DB0F0BD000041542B43E1
:106F2000495053454E443D25642C25640D0A00000C
:106F300041542B43495053454E440000DC09002086
:106F400010B514A0FCF780FC1748F9F708FC17A14E
:106F500018A0FDF76FF818A11AA0FDF76BF81BA198
:106F60001DA0FDF767F81EA120A0FDF763F821A181
:106F700024A0FDF75FF826A129A0FDF75BF82BA15F
:106F80002EA0FDF757F802202F4908700846007818
:106F900010BD00006D6F64756C655F696E6974216A
:106FA00021210D0A00000000DC0900204154453079
:106FB0000D0A00004154450041542B4350494E3FB7
:106FC0000D0A000041542B4350494E0041542B43BD
:106FD00053510D0A0000000041542B43535100004F
:106FE00041542B4347534E0D0A00000041542B439C
:106FF00047534E0041542B4349504D4F44453D307B
:107000000D0A000041542B4349504D4F44450000A8
:1070100041542B4E4554434C4F53450D0A0000003C
:1070200041542B4E4554434C4F53450041542B4E35
:1070300045544F50454E0D0A0000000041542B4E60
:1070400045544F50454E00005001002010B500201F
:1070500006490870064A01214FF47A7003F05AF885
:1070600003F096F80148007810BD000050010020A0
:10707000854100082DE9F74398B0814614460EA1DA
:1070800011A0FCF7D7FF9DF864509DF865609DF84E
:1070900066709DF867802B4601220EA104A88DE83A
:1070A000C0010394FCF702FC04A914A0FCF7C2FF82
:1070B0001BB0BDE8F083000041542B434950434CC2
:1070C0004F53453D310D0A0041542B434950434C29
:1070D0004F53450041542B4349504F50454E3D2599
:1070E000642C22544350222C2225642E25642E2504
:1070F000642E2564222C25640D0A000041542B4384
:1071000049504F50454E000070B504460120FCF731
:10711000AFFB9620FDF732FE0BA0FCF7B7FB9620E5
:10712000FDF72CFE0020FCF7A3FB25460B490120B0
:1071300001F052FC0A4802F0B9FB094802F0F8FBE2
:10714000074802F0D9FB70BD4D5154543A20436FAB
:107150006E6E65637465640D0A000000E1950008B9
:10716000F41000202DE9F84F8A4617469946DDF8BD
:1071700028800120FCF77CFB9620FDF7FFFD94A002
:10718000FCF784FB9620FDF7F9FD0020FCF770FB6F
:107190000120FCF76DFB9620FDF7F0FD394690A02D
:1071A000FCF774FB9620FDF7E9FD0020FCF760FB7F
:1071B0000120FCF75DFB9620FDF7E0FD41468EA027
:1071C000FCF764FB9620FDF7D9FD0020FCF750FB8F
:1071D00000200090BAF1000F02D0B9F1000F10D1D9
:1071E0000120FCF745FB9620FDF7C8FD88A0FCF7C1
:1071F0004DFB9620FDF7C2FD0020FCF739FBBDE8F2
:10720000F88F781CFFF776FB0646791C3046F8F7B6
:10721000B4FF3A4651463046F8F794FF0020F05547
:107220000120FCF725FB9620FDF7A8FD31467EA046
:10723000FCF72CFB9620FDF7A1FD0020FCF718FBC6
:107240004FF0000B3078632808D064280CD06528F4
:1072500007D073280BD14FF0030B09E04FF0010B5F
:1072600006E04FF0020B03E04FF0030B00E0C6E72F
:1072700000BF1EB13046FDF7D1FE00260820FFF703
:1072800039FB04467CB90120FCF7F2FA9620FDF7A1
:1072900075FD6AA0FCF7FAFA9620FDF76FFD002055
:1072A000FCF7E6FAABE7A4F800804046FFF722FBC4
:1072B0006060606878B90120FCF7DAFA9620FDF783
:1072C0005DFD5EA0FCF7E2FA9620FDF757FD002079
:1072D000FCF7CEFA93E7606842464946F8F732FF7A
:1072E000002060806946204602F0D8F80120FCF7B3
:1072F000BFFA9620FDF742FD54A0FCF7C7FA96208E
:10730000FDF73CFD0020FCF7B3FA2188606802F02D
:10731000A3FC5946204601F0F9FF78B10120FCF7A3
:10732000A7FA9620FDF72AFD53A0FCF7AFFA9620A6
:10733000FDF724FD0020FCF79BFA60E70620FFF72D
:10734000D9FA054620886188401A28802888FFF7E6
:10735000D1FAC5F802006368B4F802C003EB0C016F
:107360002A88D5F80200F8F7EDFE204601F065FB0B
:10737000BDF80000012805D0BDF800004FF6FF71F0
:10738000884217D10120FCF773FA9620FDF7F6FC2E
:10739000BDF8001040A0FCF779FA9620FDF7EEFC4E
:1073A0000020FCF765FA2A88D5F802100120FDF7C5
:1073B00037FA08E0BDF8000028B92A88D5F802108D
:1073C0000020FDF72DFA2846FDF7FCFC00BF16E76C
:1073D0006D7174745F646174615F63620A000000C0
:1073E0006D71747420746F706963206C656E67745E
:1073F000683A2025640A00006D7174742064617419
:1074000061206C656E6774683A2025640A0000008C
:107410006E6F206E6565646564206D717474207094
:1074200061636B616765210074686520746F7069C2
:10743000632069733A2025730A0000006D616C6C4B
:107440006F63206572726F72210A00007061636B56
:107450006167652066726F6D207365727665722C48
:107460002067657420726964206F66206D71747482
:1074700020686561643A0A0074686520646174611B
:107480002066726F6D207365727665722069732055
:1074900077726F6E67210A007472616E736665722F
:1074A000206461746120746F207375622064657656
:1074B0006963653A2025640A0000000070B504463F
:1074C0000120FCF7D5F99620FDF758FC05A0FCF744
:1074D000DDF99620FDF752FC0020FCF7C9F925469E
:1074E00070BD00004D5154543A20446973636F6E6F
:1074F0006E65637465640D0A0000000010B50446F3
:107500000120FCF7B5F99620FDF738FC08A0FCF740
:10751000BDF99620FDF732FC0020FCF7A9F90B48D5
:10752000006820B16FF0030008490968884710BD62
:107530004D5154543A20636F6E6E656374696E6783
:10754000206572726F720D0A000000006401002055
:107550002DE9F04105460E46012E02DA0020BDE875
:10756000F08100BF28780009C01E09284AD2DFE850
:1075700000F005363738393C3A493B00012406E033
:10758000285D00F0800008B9641C02E0641CB4426D
:10759000F6DB00BFA01CB04201DB0020DFE7204685
:1075A000641C285C07022046641C285C0743E01921
:1075B000B04201DB0020D2E73C44284600F0A5F8A9
:1075C000002804DDA01CB04203DB0020C7E7002038
:1075D000C5E7601C285C295D40EA0120BFE700BFC9
:1075E00000BF00BF00BF00BF00BF042E08DB6878EB
:1075F00000F0800020B9E878A97840EA0120AEE7E1
:107600000020ACE70020AAE72DE9F04106460D4630
:10761000002701240EE0305D00F07F00611EC1EB09
:10762000C10188400744305D00F0800008B9641C47
:1076300003E0641C2888A042EDDC00BF27442988B1
:10764000A01C814202DC0020BDE8F0812046641CC1
:10765000305C4FEA00282046641C305C40EA080891
:1076600004EB08002988884202DB00202880EBE731
:107670004444304600F049F8002806DD2988A01C63
:10768000814201DC0020DFE7A41CA74201DA0020D0
:10769000DAE72888B84202DB381B288002E0288815
:1076A000001B28803019CFE770B502460B46002535
:1076B00001210EE0505C00F07F004E1EC6EBC606B6
:1076C000B0400544505C00F0800008B9491C03E05C
:1076D000491C18888842EDDC00BF0D441E88881CB8
:1076E000864201DC002070BD0846491C105C040283
:1076F0000846491C105C044308191E88B04201DD8D
:107700000020F0E71C805018EDE701460878C0F330
:107710004100704730B502460B46002001210EE0C3
:10772000545C04F07F044D1EC5EBC505AC402044FD
:10773000545C04F080040CB9491C02E0491C9942D5
:10774000EEDB00BF084430BD0146087800097047F1
:10775000F8B506460C463046FEF722FCB0880A30E3
:10776000318A884203D93046FDF7A6FBF8BDB188BF
:10777000F0684518B0880A30B080002028700420D6
:1077800068704CA00068C5F802000420A8710020B1
:10779000E871A08A000A2872207D6872206A18B1F8
:1077A000E87940F00200E871206888B1206800782C
:1077B00070B12068F8F714FD07463A463046216854
:1077C000FCF7BAFC002807DA3046FDF775FBCDE779
:1077D0003046FDF771FBC9E7E06888B3E0680078E0
:1077E00070B3E068F8F7FCFC07463A463046E168BB
:1077F000FCF7A2FC002803DA3046FDF75DFBB5E795
:107800002069F8F7EDFC07463A4630462169FCF757
:1078100093FC002803DA3046FDF74EFBA6E7E87933
:1078200040F00400E871E06918B1E87940F0200008
:10783000E871E879217E01F0030140EAC100E871B6
:107840006068A8B16068007890B16068F8F7C8FC1B
:1078500007463A4630466168FCF76EFC002803DABA
:107860003046FDF729FB81E7E87940F08000E871B8
:10787000A068A8B1A068007890B1A068F8F7B0FC43
:1078800007463A463046A168FCF756FC002803DA62
:107890003046FDF711FB69E7E87940F04000E871F8
:1078A000002003460246012100903046FDF75EFBB2
:1078B0005CE700004D5154540000000000230360B9
:1078C000C1600282704738B504462046FEF768FB67
:1078D0000020034602460C2100902046FDF746FB9F
:1078E00038BD38B504462046FEF75AFB0020034653
:1078F00002460D2100902046FDF738FB38BD38B513
:1079000004460D462046FEF74BFB29462046FCF771
:10791000F5FB18B92046FDF7CFFA38BD0020034625
:107920000246042100902046FDF720FBF5E738B51C
:1079300004460D462046FEF733FB29462046FCF759
:10794000DDFB18B92046FDF7B7FA38BD0020034625
:107950000246072100902046FDF708FBF5E72DE9D8
:10796000F84F04460D4617461E46DDE90BA9DDF823
:1079700028802046FEF714FB0DB1287820B9204658
:10798000FDF79AFABDE8F88F2846F8F729FC8346F8
:107990005A4629462046FCF7CFFB002803DA20464A
:1079A000FDF78AFAEEE7B8F1000F0ADD0021204664
:1079B000FCF7A4FBA9F8000030B92046FDF77CFADB
:1079C000E0E70020A9F80000A0883044218A88421E
:1079D00003DD2046FDF770FAD4E7A288E168881835
:1079E00032463946F8F7AEFBA0883044A0804346C3
:1079F000002203212046CDF800A0FDF7B7FAC1E729
:107A000038B504460D462046FEF7CAFA29462046F8
:107A1000FCF774FB18B92046FDF74EFA38BD00207C
:107A200003460246052100902046FDF79FFAF5E740
:107A300038B504460D462046FEF7B2FA29462046E0
:107A4000FCF75CFB18B92046FDF736FA38BD00207C
:107A500001230246062100902046FDF787FAF5E74C
:107A600070B504460120FBF703FF9620FDF786F969
:107A700005A0FBF70BFF9620FDF780F90020FBF730
:107A8000F7FE254670BD00004D5154543A20507504
:107A9000626C69736865640D0A0000002DE9FC41A1
:107AA00005460F462E46746A3149304600F040FFC5
:107AB0003049304600F048FF2F49304600F050FF73
:107AC0000120FBF7D5FE9620FDF758F92BA0D4E94D
:107AD0000212FBF7DBFE9620FDF750F90020FBF7C2
:107AE000C7FEA08D82B204F13800616AFFF7E6FE9E
:107AF00004F13800E169FFF72BFE6063616B0868F1
:107B0000FFF722FE2065626B91881068FFF720FD69
:107B10004C2108530520C4F8A800606B8088ADF89C
:107B20000000606B006801900120FBF7A1FE962029
:107B3000FDF724F94C20025B19A0216DFBF7A6FE8E
:107B40009620FDF71BF90020FBF792FEB4F8A80081
:107B500083B23046DDE9001200F00EFF00216163C0
:107B60000C2084F8B0002046FAF75CFEBDE8FC81EA
:107B7000C57B00082D7C0008518300084D515454EA
:107B80003A20436F6E6E656374656420746F206283
:107B9000726F6B65722025733A25640D0A00000030
:107BA0004D5154543A2053656E64696E672C2074AD
:107BB0007970653A2025642C2069643A2025303498
:107BC000580D0A002DE9F04105460F462E46746A0D
:107BD0000120FBF74DFE9620FDF7D0F80BA0FBF738
:107BE00055FE9620FDF7CAF80020FBF741FE06205F
:107BF00084F8B000D4F8800018B12046D4F8801082
:107C000088472046FAF70EFEBDE8F0815443503A0B
:107C100020446973636F6E6E65637465642063618D
:107C20006C6C6261636B0D0A000000002DE9FE4F71
:107C300083460E460120FBF71BFE9620FDF79EF8BB
:107C40003188FEA0FBF722FE9620FDF797F8002072
:107C5000FBF70EFECDF808B0DDF808B0DBF82440E5
:107C60003088B0F5806F01DC308880B90120FBF7E7
:107C7000FFFD9620FDF782F8F8A0FBF707FE96209F
:107C8000FDF77CF80020FBF7F3FDBDE8FE8F638E67
:107C9000D4F820C00CEB030032887168F8F752FA70
:107CA000608E31880844608600BF608E01280ED146
:107CB000FBF7DEFD9620FDF761F8EFA0FBF7E6FD90
:107CC0009620FDF75BF80020FBF7D2FDDDE7618E23
:107CD000206AFFF71FFD20860120FBF7C9FD9620D3
:107CE000FDF74CF8218EEFA0FBF7D0FD9620FDF7B5
:107CF00045F80020FBF7BCFD618E206A01F0ACFF67
:107D0000218E608E81420FDD0120FBF7B1FD9620B0
:107D1000FDF734F8E8A0FBF7B9FD9620FDF72EF843
:107D20000020FBF7A5FDB0E7206AFFF70DFD00F08E
:107D3000FF09206A0178C1F3410500BF218E206A46
:107D4000FFF706FC07460120FBF792FD9620FDF7A2
:107D500015F8208ECDE9007094F8B0102B464A46F5
:107D6000DA48FBF793FD9620FDF708F80020FBF7B3
:107D70007FFD94F8B0000C2802D00F2832D132E0F9
:107D8000B9F1020F2ED1206D012812D00120FBF78E
:107D90006FFD9620FCF7F2FFCDA0FBF777FD962054
:107DA000FCF7ECFF0020FBF763FD206800F09CFD72
:107DB00018E00120FBF75CFD9620FCF7DFFFCAA06E
:107DC000D4E90212FBF762FD9620FCF7D7FF0020F2
:107DD000FBF74EFD0F2084F8B000E06F10B1204695
:107DE000E16F884721E1A9F103000B281DD2DFE8EC
:107DF00000F0347B92B1D01C061C1DE7FD00206D05
:107E0000082806D14C20005BB84202D10120FBF7C4
:107E10002FFD9620FCF7B2FFBAA0FBF737FD9620A6
:107E2000FCF7ACFF0020FBF723FDFCE0206D0A28E7
:107E300006D14C20005BB84202D10120FBF718FDAF
:107E40009620FCF79BFFB7A0FBF720FD9620FCF7E0
:107E500095FF0020FBF70CFDE5E0012D06D139462A
:107E600004F13800FFF74BFD606307E0022D05D1F8
:107E7000394604F13800FFF7C3FD6063012D01D0DE
:107E8000022D27D10120FBF7F3FC9620FCF776FFAB
:107E90002946ACA0FBF7FAFC9620FCF76FFF002008
:107EA000FBF7E6FC606B8288016804F1B400FAF726
:107EB00012FF401C70B90120FBF7DAFC9620FCF79A
:107EC0005DFFA8A0FBF7E2FC9620FCF757FF00201F
:107ED000FBF7CEFC218E206A01F0BEFE228E2046EA
:107EE000216AFCF7A8FF9EE0206D032812D14C20E8
:107EF000005BB8420ED10120FBF7BAFC9620FCF7DC
:107F00003DFF9DA0FBF7C2FC9620FCF737FF002049
:107F1000FBF7AEFC87E0394604F13800FFF788FD37
:107F20006063606B8288016804F1B400FAF7D3FEE5
:107F3000401C70B90120FBF79BFC9620FCF71EFF4C
:107F400088A0FBF7A3FC9620FCF718FF0020FBF7A6
:107F50008FFC68E0394604F13800FFF7E8FC606305
:107F6000606B8288016804F1B400FAF7B4FE401C2B
:107F700070B90120FBF77CFC9620FCF7FFFE79A08E
:107F8000FBF784FC9620FCF7F9FE0020FBF770FC61
:107F900049E0206D032812D14C20005BB8420ED17D
:107FA0000120FBF765FC9620FCF7E8FE81A0FBF7BB
:107FB0006DFC9620FCF7E2FE0020FBF759FC32E056
:107FC00004F13800FFF78DFC6063606B8288016804
:107FD00004F1B400FAF77FFE401C80B90120FBF7E2
:107FE00047FC9620FCF7CAFE5EA000E008E0FBF725
:107FF0004DFC9620FCF7C2FE0020FBF739FC12E096
:108000000120FBF735FC9620FCF7B8FE78A0FBF7C3
:108010003DFC9620FCF7B2FE0020FBF729FC012076
:10802000C4F8AC0000BF00BF00BF00BF618E208E4F
:10803000081A1FFA80F8A4F83280E9E05443503A55
:1080400020646174612072656365697665642025CA
:10805000642062797465730D0A00000072656365BF
:10806000697665206C656E67746820697320696E37
:1080700076616C69642E0A006E6F7420656E6F7590
:108080006768206461746120666F72207265616444
:10809000207061636B616765206C656E6774682E24
:1080A0000A2100006D657373616765206C656E67FA
:1080B00074683A25640A00006E6F7420656E6F75EF
:1080C000676820646174612E0A00000090AA0008AD
:1080D0004D5154543A20496E76616C696420706148
:1080E000636B65740D0A00004D5154543A20436F80
:1080F0006E6E656374656420746F2025733A256421
:108100000D0A00004D5154543A2053756273637246
:10811000696265207375636365737366756C0D0AB8
:10812000000000004D5154543A20556E537562734F
:108130006372696265207375636365737366756CDA
:108140000D0A00004D5154543A2051756575652053
:10815000726573706F6E736520516F533A2025649A
:108160000D0A00004D5154543A2051756575652033
:1081700066756C6C0D0A00004D5154543A207265BE
:10818000636569766564204D5154545F4D53475F74
:10819000545950455F50554241434B2C2066696EFF
:1081A00069736820516F5331207075626C69736810
:1081B0000D0A00004D5154543A207265636569768A
:1081C00065204D5154545F4D53475F545950455F9E
:1081D000505542434F4D502C2066696E697368209C
:1081E000516F5332207075626C6973680D0A00001C
:1081F00072656365697665206120686561727420C7
:108200006265617420726573706F6E7365210A0018
:108210000120FBF72DFB9620FCF7B0FD618E2AA014
:10822000FBF734FB9620FCF7A9FD0020FBF720FBB1
:108230000120FBF71DFB9620FCF7A0FD218E2EA050
:10824000FBF724FB9620FCF799FD0020FBF710FBC1
:108250000120FBF70DFB9620FCF790FD30A0FBF70B
:1082600015FB9620FCF78AFD0020FBF701FB218E11
:10827000206A01F0F1FCB8F1000F20DD4FF0000A98
:1082800000BF0AE0608EA0EB08005044216A095C40
:10829000206A00F80A100AF1010AC245F2DB012047
:1082A000FBF7E6FA9620FCF769FD21A0FBF7EEFA52
:1082B0009620FCF763FD0020FBF7DAFAF5E4204690
:1082C000FAF7B0FA00BFE0E4636C69656E742D3EA6
:1082D0006D7174745F73746174652E6D6573736111
:1082E00067655F6C656E6774685F72656164203D89
:1082F0002025640A00000000636C69656E742D3EE1
:108300006D7174745F73746174652E6D65737361E0
:1083100067655F6C656E677468203D2025640A00A0
:10832000746865207061636B6167652069730A001A
:1083300047657420616E6F74686572207075626C39
:108340006973686564206D6573736167650D0A0004
:108350002DE9F04105460E462F467C6A06BB0120FA
:10836000FBF786FA9620FCF709FD1BA0FBF78EFAB7
:108370009620FCF703FD0020FBF77AFA0020C4F8F2
:10838000A80094F8B0000F2821D1206D03281ED139
:10839000D4F88400D8B12046D4F88410884716E079
:1083A000701CA0B90120FBF763FA9620FCF7E6FCED
:1083B0000DA0FBF76BFA9620FCF7E0FC0020FBF722
:1083C00057FA0020C4F8A800062084F8B000204620
:1083D000FAF728FABDE8F0815443503A2053656E0D
:1083E00074204F4B0D0A00005443503A2073656EC1
:1083F00074206661696C6564210000007CB50546E7
:108400002C460120FBF734FA9620FCF7B7FC94F8D1
:10841000B020634963A0FBF739FA9620FCF7AEFC65
:108420000020FBF725FA94F8B0000F2862D154F829
:108430009C0F401C206054F89C19E06940698142FF
:1084400057D9D4F8AC0010B9062084F8B000012048
:10845000FBF70EFA9620FCF791FC54A0D4E9021227
:10846000FBF714FA9620FCF789FC0020FBF700FAD2
:1084700004F13800FFF727FA60630C212165616B76
:108480000868FFF761F92065626B91881068FFF753
:108490005FF84C2108530520C4F8A800606B808861
:1084A000ADF80000606B006801900120FBF7E0F977
:1084B0009620FCF763FC4C20025B47A0216DFBF784
:1084C000E5F99620FCF75AFC0020FBF7D1F9B4F847
:1084D000A8108BB22068DDE9001200F04DFA0021EF
:1084E00061630020C4F89C00C4F8AC002046FAF791
:1084F00099F94CE094F8B000062822D10120FBF74E
:10850000B7F99620FCF73AFC54F8A02F24493BA079
:10851000FBF7BCF99620FCF731FC0020FBF7A8F92B
:108520002068401C206054F8A00905282FD900209D
:10853000C4F8A000072084F8B0002046FAF772F9CA
:1085400025E094F8B000082821D10120FBF790F92C
:108550009620FCF713FC54F8A42F11492FA0FBF729
:1085600095F99620FCF70AFC0020FBF781F92068BA
:10857000401C206054F8A409142808D9092084F864
:10858000B0000020C4F8A4002046FAF74BF9D4F854
:10859000A80020B1D4F8A800401EC4F8A8007CBDF3
:1085A00039A6000825732C2025640A000D0A4D51B8
:1085B00054543A2053656E64206B656570616C6934
:1085C0007665207061636B657420746F2025733A43
:1085D0002564210D0A0000004D5154543A20536582
:1085E0006E64696E672C20747970653A2025642C5E
:1085F0002069643A20253034580D0A0025732C2058
:10860000636C69656E742D3E7265636F6E6E656333
:10861000745469636B3A25640A00000025732C20AA
:10862000636C69656E742D3E636F6E6E6563745422
:1086300069636B3A25640A0000B50246FDF79EFDAA
:1086400020B1100AD1B240EA012000BD1046FCE77B
:1086500000B50246FDF792FD58B1100E02F47F01FD
:1086600040EA112002F47F4140EA012040EA026022
:1086700000BD1046FCE718B50446FDF77FFD30B19C
:1086800000940098FFF7E4FF0090009818BD204682
:10869000FCE72DE9F04106460F46FF240025FDF7D3
:1086A0006DFD00283DD007EA0460020E002107EAB4
:1086B000044042EA10200943002307EA042C43EA5D
:1086C0000C220B4640EA020143EA1C6004EA07035D
:1086D0004FEA036C41EA0C0240EA1323290641EAFF
:1086E000142106EA046C3940080240EA1C6042EAA0
:1086F0000C210343280440EA144006EA04423840AF
:10870000000640EA122C41EA026043EA0C0106EA44
:10871000042241EA022106EA040241EA0261BDE8BC
:10872000F08130463946FAE77CB504460D46FDF740
:1087300025FD58B1CDE90045DDE900211046FFF7E0
:10874000A8FFCDE90001DDE900017CBD20462946F6
:10875000FBE700002DE9FF4180460E461F4B0FCB83
:108760008DE80F004FF0FF370025344600E0641C11
:1087700020780D28FBD020780A28F8D0002509E0C1
:108780005DF825102046F7F703FD08B16FB203E04E
:10879000681CC5B2042DF3D300BF37B1012F08D038
:1087A000022F0AD0032F10D10BE001200C490870D2
:1087B0000CE001200A49087008E00120084908700F
:1087C00004E001200649087000E000BF00BF044833
:1087D000007840B204B0BDE8F0810000F8A40008C1
:1087E0005101002010B50024FDF7FAFB04460C2CC3
:1087F00001DD012010BD0020FCE770B504460D46E8
:108800001646324629462046FEF774F970BD000030
:108810002DE9FE4380460E46204A07CA8DE8070030
:108820004FF0FF370025344600E0641C20780D2807
:10883000FBD020780A28F8D0002509E05DF8251043
:108840002046F7F7A5FC08B16FB203E0681CC5B27B
:10885000032DF3D300BF27B1012F09D0022F15D16B
:108860000DE001200E49087003200E4908700EE04B
:1088700001200B49087003200A49087007E0012015
:108880000749087003200749087000E000BF00BFD7
:108890000348007840B2BDE8FE830000ECA4000865
:1088A00051010020500100202DE9F0410446884686
:1088B00066682789002500BF09E00A4850F82500AE
:1088C00020B96582074840F8254002E06D1C0A2D5A
:1088D000F3DB00BF608A3A463146FEF7CBFBBDE8CA
:1088E000F08100008C1200200146002000BF0CE047
:1088F0004A8A084B53F820305B8A9A4204D10022FE
:10890000044B43F8202002E0401C0A28F0DB00BFA3
:10891000704700008C12002070B504460D4665615A
:10892000608A024901F06AF870BD0000859E000867
:1089300070B504460D4625620249002001F064F836
:1089400070BD0000299F000870B504460D46A56162
:108950000249002001F05EF870BD0000B19F0008E0
:1089600070B504460D46E5610249002001F058F853
:1089700070BD000015A000087FB504461D4601200B
:10898000FAF776FF9620FCF7F9F90B490BA0FAF7F6
:108990007DFF9620FCF7F2F90020FAF769FFBDF899
:1089A0000410029801F058F9BDF804200020029943
:1089B000FEF790FA7FBD000091A6000825732C7485
:1089C00063702073656E640A0000000010B5082013
:1089D000FDF790FF10BD000000EB4002024B03EBDF
:1089E0008202916070470000B00F002000EB40024F
:1089F000024B03EB8202516070470000B00F002071
:108A000070B505460E460820FDF774FF04460CB904
:108A1000002070BD258066802088FDF76BFF6060B8
:108A2000606820B92046FCF7F9FA0020F1E72188B8
:108A30006068F7F7A2FB2046EBE710B5044604B9DF
:108A400010BD606810B16068FCF7E8FA2046FCF7DA
:108A5000E5FA00BFF4E700002DE9F04397B00446C3
:108A60000120FAF705FF9620FCF788F953A0FAF7E2
:108A70000DFF9620FCF782F90020FAF7F9FE01209D
:108A8000FAF7F6FE9620FCF779F954A0FAF7FEFE05
:108A90009620FCF773F90020FAF7EAFE0CB1534870
:108AA000046053A000F004F90546B5B90120FAF7B7
:108AB000DFFE9620FCF762F952A0FAF7E7FE962057
:108AC000FCF75CF90020FAF7D3FE6FF0030047498A
:108AD0000968884717B0BDE8F08316AA12A928468E
:108AE000FBF7EAFEA0B10120FAF7C2FE9620FCF7E0
:108AF00045F94DA0FAF7CAFE9620FCF73FF9002091
:108B0000FAF7B6FE6FF00300384909688847E1E7D5
:108B10004DA000F0CDF880464046F7F7A8FB81460F
:108B20004A464DA14D48FAF7C1FEFDF7EBF9012386
:108B300012A94B48169AF9F767FD4AA000F0B8F859
:108B400007463846F7F74CFB461C3246394602A822
:108B5000F7F7F8FA01201E2102AB47A2CDE9001079
:108B60003E493F48F9F7C0FC0120FAF781FE962004
:108B7000FCF704F9394941A0FAF788FE9620FCF782
:108B8000FDF80020FAF774FE44493548F9F77DFDF9
:108B900043493348F9F77EFD42493148F9F77DFDF5
:108BA00041492F48F9F773FD40492D48F9F76AFD0F
:108BB0002B48F9F7DFFB00BF8CE7000050414E4423
:108BC0004F3A20626567696E206163636573732045
:108BD000636C6F75642E2E2E0A0000006265666F4E
:108BE0007265206163636573733A0A006401002053
:108BF00070616E646F5F6163636573735F6164640A
:108C0000720000006E6F206163636573732073658B
:108C100072766572206164647265737320666F7525
:108C20006E642E2E2E0A000077726F6E67206163CD
:108C30006365737320736572766572206164647214
:108C40006573732E2E2E0A0070616E646F5F64650B
:108C5000766963655F69640025780000E010002094
:108C60001010002070616E646F5F616363657373E1
:108C70005F746F6B656E00000000000061636365E8
:108C80007373207374725F6465766963655F69648A
:108C90005F6865783A25730A0000000009710008D2
:108CA000BD740008617A000865710008FD74000851
:108CB00070B505462846FCF713F9044614B104F1D3
:108CC000240070BD0020FCE72DE9F04106460F4668
:108CD0003046FCF705F90546C5B16022394605F175
:108CE0002400F7F767FA0120FAF7C2FD9620FCF797
:108CF00045F805F1240231461AA0FAF7C7FD96207F
:108D0000FCF73CF80020FAF7B3FD26E08420FDF7DD
:108D1000F1FD044620223146201DF7F74BFA602270
:108D2000394604F12400F7F745FA15480068206039
:108D3000134804600120FAF79BFD9620FCF71EF80B
:108D400004F1240231460FA0FAF7A0FD9620FCF7AB
:108D500015F80020FAF78CFD00BF00F085FE012019
:108D6000BDE8F0816B6579202573207570646174AE
:108D700065642C76616C75653A25730A0000000005
:108D8000A80100206B6579202573206372656174EA
:108D900065642E2E2E2C2076616C7565202573203F
:108DA0000A0000002DE9F041AEB004460120FAF7B8
:108DB0005FFD9620FBF7E2FF48A0FAF767FD9620DB
:108DC000FBF7DCFF0020FAF753FD0CB149480460C3
:108DD0000025002648A0FFF76BFF05464AA0FFF7D5
:108DE00067FF064605B1B6B90120FAF741FD9620A6
:108DF000FBF7C4FF49A0FAF749FD9620FBF7BEFF39
:108E00000020FAF735FD6FF001003A4909688847FC
:108E10002EB0BDE8F0812846F7F729FA07464C49FD
:108E200003C9CDE92C012D974949083103C9CDE982
:108E30002A012B964649103103C9CDE92801182291
:108E40004349183122A8F7F77DF92CA823902AA9C5
:108E500022A8C16028A941613D49303103C9CDE94B
:108E6000200122A821904FF48070FDF743FD39497D
:108E700008604FF480720846016820A800F002FAEA
:108E800080460120FAF7F4FC9620FBF777FF314883
:108E9000016831A0FAF7FAFC9620FBF76FFF00207B
:108EA000FAF7E6FC80216846F7F767F933A23BA1A1
:108EB0006846FAF7FBFC414A264801686846FFF716
:108EC0009CFC2448006830B122480068FCF7A6F8F2
:108ED00000202049086000BF9AE7000062656769CA
:108EE0006E206C6F67696E206465766963652E2EEF
:108EF0002E0A00007001002070616E646F5F64656F
:108F0000766963655F69640070616E646F5F646554
:108F1000766963655F736563726574006C6F67691A
:108F20006E206661696C65642021206465766963E2
:108F30006520686173206E6F74206265656E2072B3
:108F400065676973746572642E2E2E0A0000000036
:108F500090A5000874010020646576696365206C43
:108F60006F67696E20726571756573743A3A3A0A73
:108F700025730A28656E64290A00000068747470FD
:108F80003A2F2F3232322E3137352E3132392E31BF
:108F900039343A31383038380000000025732F76E4
:108FA000312F646576696365732F61757468656ECA
:108FB0007469636174696F6E000000007955000880
:108FC0002DE9F041BAB004460120FAF751FC962091
:108FD000FBF7D4FE4EA0FAF759FC9620FBF7CEFE25
:108FE0000020FAF745FC0CB151480460002500262A
:108FF000002750A0FFF75CFE054652A0FFF758FE81
:10900000064655A0FFF754FE074636A8FCF774F84D
:1090100000208DF8E7000120FAF72AFC9620FBF7E4
:10902000ADFE36A951A0FAF731FC9620FBF7A6FE5B
:109030000020FAF71DFC524903C9CDE9340150491B
:10904000083103C9CDE9320136A833904C491031BB
:1090500003C9CDE930014A49183103C9CDE92E01D0
:109060004749203103C9CDE92C0128224449283140
:1090700022A8F7F767F834A8239032A922A8C16084
:1090800030A941612EA9C1612CA941623C495031EE
:1090900003C9CDE9200122A821904FF48070FDF78B
:1090A00029FC384908604FF480720846016820A8FE
:1090B00000F0E8F880460120FAF7DAFB9620FBF78B
:1090C0005DFE3048016830A0FAF7E0FB9620FBF720
:1090D00055FE0020FAF7CCFB80216846F7F74DF8E3
:1090E00033A23BA16846FAF7E1FB404A25480168F4
:1090F0006846FFF782FB2348006830B121480068CA
:10910000FBF78CFF00201F4908603AB0BDE8F081F2
:1091100050414E444F20626567696E2072656769F1
:1091200073746572206465766963652E2E2E0A005D
:109130007801002070616E646F5F646576696365B5
:109140005F69640070616E646F5F64657669636512
:109150005F7365637265740070616E646F5F6465F0
:10916000766963655F6B6579000000006465766908
:1091700063655F73657269616C3A25730A0000006C
:10918000C8A500087C0100206465766963652072CB
:109190006567697374657220726571756573743A79
:1091A0003A3A0A25730A28656E64290A000000000D
:1091B000687474703A2F2F3232322E3137352E3197
:1091C00032392E3139343A31383038380000000025
:1091D00025732F76312F646576696365732F726509
:1091E00067697374726174696F6E000005580008D6
:1091F00010B500F007F802490120FFF7F7FB10BD9A
:10920000CD97000810B50120FAF732FB9620FBF746
:10921000B5FD12A0FAF73AFB9620FBF7AFFD002050
:10922000FAF726FB002014490870FDF771FA00F0E8
:109230009BFB41F28830114908800120887010485A
:1092400048600220C870084600F030FB0B4800F070
:109250006FFB0A4800F050FB10BD000050414E4427
:109260004F206761746577617920696E69746961FF
:109270006C2E2E2E2E0A00008001002000110020EE
:10928000854E000870B592B005460C4616461CB9CE
:109290004FF0FF3012B070BD0D4804600D480660FD
:1092A00000200D49086000956846FDF771F90B48EC
:1092B0000F9000BF6846FDF7BDF80028FAD10449B9
:1092C0000968054A1268885403480068E2E700000C
:1092D00084010020880100208C0100201162000818
:1092E00001460878074A1268904201D10020704771
:1092F0000A78501C087002EB4200034A02EB80001F
:10930000F5E70000A4010020CC1100202DE9FE4368
:1093100004460E466068618845186068218800EB45
:1093200001082F463846FBF79FFA18B14FF0FF307F
:10933000BDE8FE831935454511D90120FAF798FAA1
:109340009620FBF71BFD10A0FAF7A0FA9620FBF77A
:1093500015FD0020FAF78CFA4FF0FF30E8E720887F
:109360006188401A83B2324639466846FCF7A6FD4A
:109370000C3D00982860019868600298A860608899
:109380000D3060800020D3E7496E636F72726563B1
:1093900074206465636F646520627566666572201B
:1093A0006C656E6774682E0A000000002DE9F041BC
:1093B0008AB004460D466068618846186068218856
:1093C00000EB0108374606F10C000646404513D96C
:1093D0000120FAF74DFA9620FBF7D0FC1FA0FAF710
:1093E00055FA9620FBF7CAFC0020FAF741FA4FF035
:1093F000FF300AB0BDE8F081788828802888FFF720
:109400001BF92880F888ADF80600BDF80600FFF7C4
:1094100013F9ADF80600694603A8FCF7C5FD88B14D
:109420000120FAF725FA9620FBF7A8FC14A0FAF71A
:109430002DFA9620FBF7A2FC0020FAF719FA4FF05C
:10944000FF30D6E7193E192203A93046F6F77AFE17
:1094500060880D3860800020CBE70000496E636FA4
:10946000727265637420656E636F646520627566F1
:10947000666572206C656E6774682E0A00000000D5
:10948000496E697420706462696E20686561646504
:1094900072206661696C65642E0A000070B505462D
:1094A0000C4668681930698846188EB90120FAF7A9
:1094B000DFF99620FBF762FC09A0FAF7E7F996209E
:1094C000FBF75CFC0020FAF7D3F94FF0FF3070BDDA
:1094D000308820802088FFF7AFF820800020F6E752
:1094E000737562646576696365206E756C6C0A00DD
:1094F0000FB410B5342202A90C48F6F723FE98B930
:109500000120FAF7B5F99620FBF738FC08A0FAF726
:10951000BDF99620FBF732FC0020FAF7A9F94FF0CD
:10952000FF3010BC5DF814FB0020FAE70C1100209E
:1095300070616E646F5F70726F746F636F6C5F6980
:109540006E6974206661696C65642E0A0000000013
:1095500073B5044660681930618845188DB90120DB
:10956000FAF786F99620FBF709FC13A0FAF78EF9B3
:109570009620FBF703FC0020FAF77AF94FF0FF3052
:109580007CBD0120FAF774F99620FBF7F7FBBDF8D4
:1095900004100DA0FAF77AF99620FBF7EFFB0020F4
:1095A000FAF766F9BDF80400FFF746F80190BDF838
:1095B000040028800020E3E77375626465766963C0
:1095C00065206E756C6C0A00736574207375625F3C
:1095D0006465766963655F69642025640A0000003C
:1095E0002DE9FF4106460D460120FAF741F9962084
:1095F000FBF7C4FB4CA0FAF749F99620FBF7BEFB3A
:109600000020FAF735F9002400270020039005F127
:109610000D0087B20D213846FFF7F2F90446606865
:1096200088B90120FAF724F99620FBF7A7FB4549F2
:1096300045A0FAF72BF99620FBF7A0FB0020FAF7DC
:1096400017F9BDE8FF816168628888182A463146AB
:10965000F6F778FD03A92046FFF7A8FE78B10120B0
:10966000FAF706F99620FBF789FB3CA0FAF70EF90A
:109670009620FBF783FB0020FAF7FAF8E1E70121D7
:109680002046FFF765FF2188606800F0E5FABDF825
:109690000C00012804D0022806D003280CD107E0D2
:1096A00036A0006802901AE035A00068029016E02B
:1096B00034A00068029012E00120FAF7D9F8962051
:1096C000FBF75CFB30A0FAF7E1F89620FBF756FBBE
:1096D0000020FAF7CDF82046FFF7AFF9B1E700BF59
:1096E0002E4890F8B0000F280AD100200121CDE9C2
:1096F00000102388626802A92848F8F7D1FF0EE01D
:109700000120FAF7B5F89620FBF738FB24A0FAF70A
:10971000BDF89620FBF732FB0020FAF7A9F82046A7
:10972000FFF78BF900BF8CE770616E646F5F707537
:10973000626C6973685F646174615F6368616E6EB7
:10974000656C310074A5000825733A6D616C6C6F0F
:1097500063206661696C65642E0A000070616E6446
:109760006F5F70726F746F636F6C5F656E636F6451
:1097700065206572726F722E0A000000630000009F
:1097800065000000730000006572726F72207061E6
:10979000796C6F616420747970650A001010002084
:1097A0004D515454207374617465206973206E6F39
:1097B00074206176616961626C6520666F722070E9
:1097C00075626C6973682F6E000000002DE9F0412E
:1097D00007460D460FB9BDE8F0810120FAF748F8B9
:1097E0009620FBF7CBFA22A0FAF750F89620FBF769
:1097F000C5FA0020FAF73CF82946384600F02CFA62
:109800000620FDF777F8044625802846FDF772F814
:10981000C4F80200D4F802002A463946F6F792FC52
:109820002046FBF7CDFC0646012E05D0032E07D1BE
:109830002046FBF74DFA14E02046FBF7D7F910E07D
:109840000120FAF715F89620FBF798FA314610A098
:10985000FAF71CF89620FBF791FA0020FAF708F8BF
:1098600000BF00BF2046FBF7ADFA00BFB3E7000022
:10987000737562646576697665207265636569767D
:10988000652061207061636B6167653A200A0000A2
:10989000756E7375706F727465642070616C6F6142
:1098A000642074797065203A2025640010B5044660
:1098B000E078012805D109480460204600F0E6FB65
:1098C0000AE0E078022804D10548046000F070FC4A
:1098D00002E004A0F9F7DAFF10BD0000AC0100209F
:1098E000B001002077726F6E672074696D65722019
:1098F0006E6F210A0000000010B50446E0780128D0
:1099000002D100F0F7FB08E0E078022802D100F075
:1099100087FC02E001A0F9F7B9FF10BD77726F6E06
:10992000672074696D6572206E6F210A0000000067
:1099300010B50446E078012802D100F0E3FB08E00E
:10994000E078022802D100F073FC02E001A0F9F7F0
:109950009DFF10BD77726F6E672074696D65722010
:109960006E6F210A0000000010B502490020FFF7C9
:109970003DF810BD6DA30008002001467047014668
:10998000C86808B900207047C868401EC86001F167
:109990001A00CA68805CF6E770B50E4804680CB916
:1099A000002070BDA66846B92568002009490860F6
:1099B0002046FBF733FB2846F3E725680548066099
:1099C0000020044909684860A0602046FBF726FB98
:1099D0002846E6E720000020024602F11A00D3687C
:1099E000C154D068401CD06000201076D0680A288E
:1099F00001DA012070470020FCE70000014A1160F5
:109A00007047000038000020014A116070470000D4
:109A100044000020014A116070470000400000200F
:109A2000014A1160704700003C00002007B50A4859
:109A300000680F2800DD0EBD074801680068401C63
:109A4000054A106001EB4100044901EB80009DE8EC
:109A50000E000EC000BFEEE7A4010020CC110020D4
:109A600010B500F061F810BD38B50120F9F700FF1E
:109A70009620FBF783F91BA0F9F708FF9620FBF768
:109A80007DF90020F9F7F4FE002000901C480468DE
:109A900011E09DF8001001EB41110C2202EB810155
:109AA00088B284222146F6F7C7FD9DF80000401CCD
:109AB000C0B200902468002CEBD1012269460B2033
:109AC000F6F7BAFD0120F9F7D3FE9620FBF756F919
:109AD0000CA0F9F7DBFE9620FBF750F90020F9F710
:109AE000C7FE38BD736176696E672064617461205A
:109AF000746F20666C6173682E2E2E0A00000000C1
:109B0000A8010020646F6E652E2E2E0A0000000052
:109B100070B504462046F6F763FB85B22946204619
:109B2000F9F784FE70BD00002DE9F0410020FAF73E
:109B30003BFF044684B90120F9F79AFE9620FBF713
:109B40001DF92CA0F9F7A2FE9620FBF717F90020CB
:109B5000F9F78EFEBDE8F0810025FAF77FFF804619
:109B600030E0FAF785FF06467EB90120F9F780FE5E
:109B70009620FBF703F926A0F9F788FE9620FBF75D
:109B8000FDF80020F9F774FEE4E73046696888477D
:109B9000297832462046FAF705FA074677B10120C0
:109BA000F9F766FE9620FBF7E9F821A0F9F76EFEBB
:109BB0009620FBF7E3F80020F9F75AFE3046FBF752
:109BC00021F900BF4046FFF78BFB051EC9D1404677
:109BD000FBF711F92288D4F802100120FAF7EEFD04
:109BE0002188D4F8020000F037F82046FBF7EAF8A5
:109BF00000BFAFE7637265617465206461746120C2
:109C00007061636B616765206572726F720A000034
:109C100043726561746520706172616D7320626C5E
:109C20006F636B206661696C65642E0A000000003A
:109C30006164645F6E6578745F70726F7065727472
:109C400079206661696C65642E0000000149087026
:109C5000704700005001002070B505460E460024F4
:109C60000120F9F705FE9620FBF788F8314617A08A
:109C7000F9F70CFE9620FBF781F80020F9F7F8FDC4
:109C800000BF10E00120F9F7F3FD9620FBF776F80E
:109C9000295D17A0F9F7FAFD9620FBF76FF8002071
:109CA000F9F7E6FD641CB442ECDB0120F9F7E0FDB6
:109CB0009620FBF763F810A0F9F7E8FD9620FBF774
:109CC0005DF80020F9F7D4FD70BD00005061636BB2
:109CD000616765206C656E6774683A2025640A6365
:109CE0006F6E74656E742069733A200A000000007C
:109CF00025303278200000000A00000070B50546CB
:109D00000E4600240120F9F7B3FD9620FBF736F844
:109D1000314617A0F9F7BAFD9620FBF72FF800207F
:109D2000F9F7A6FD00BF10E00120F9F7A1FD96208C
:109D3000FBF724F8295D17A0F9F7A8FD9620FBF79B
:109D40001DF80020F9F794FD641CB442ECDB0120FF
:109D5000F9F78EFD9620FBF711F810A0F9F796FDA4
:109D60009620FBF70BF80020F9F782FD70BD00008C
:109D70005061636B616765206C656E6774683A203B
:109D800025640A636F6E74656E742069733A200AE5
:109D90000000000025303278200000000A0000009A
:109DA00002E04268521C4260D0E901239A4206DA7E
:109DB000D0E90023D15C2029F3D00A29F1D07047E3
:109DC0002DE9FE4381460E46274A07CA8DE8070063
:109DD0004FF0FF370025344600E0641C20780D2842
:109DE000FBD020780A28F8D0002509E05DF825107E
:109DF0002046F6F7CDF908B16FB203E0681CC5B292
:109E0000032DF3D300BF27B1012F1BD0022F24D184
:109E100022E016A12046F6F7BBF904460C34204692
:109E2000F6F718FA8046B8F1000F07D1134800681A
:109E300020B100210846114A1268904701201049BC
:109E400008700BE04FF0FF3100200C4A1268904779
:109E500001200B49087001E000E000BF00BF084886
:109E6000007840B2BDE8FE8308A500082B434950A6
:109E70004F50454E3A20312C0000000038000020A1
:109E80005101002070B504460D460E490EA0F9F7A9
:109E9000FDFC2E46601C18B913A0F9F7F7FC10E082
:109EA000174850F8240060B1154850F82400406964
:109EB00038B1134951F8240051F824104A69314649
:109EC000904770BD4EA6000825732C6465627567C7
:109ED0003A6E657420636F6E6E6563742063616CA7
:109EE0006C6261636B0A00006D6F64756C65206362
:109EF000616C6C6261636B206572726F72210A0023
:109F00008C12002070B504460D460648006828B142
:109F10004FF0FF310020034A126890474FF0FF30A6
:109F200070BD00004400002070B504460D460E4987
:109F30000EA0F9F7ABFC601C18B913A0F9F7A6FC4A
:109F400010E01A4850F8240060B1184850F8240076
:109F5000006A38B1154951F8240051F824100A6AF2
:109F60002946904770BD000077A6000825732C6431
:109F7000656275673A6E657420646973636F6E65B8
:109F80006374206F6B0A00006D6F64756C652064EC
:109F90006973636F6E6E6563742063616C6C62617C
:109FA000636B206572726F72210A00008C120020B0
:109FB0007CB504460D4616460195ADF80060601C60
:109FC00018B90BA0F9F762FC10E0114850F8240012
:109FD00060B10F4850F82400806938B10C4951F83D
:109FE000240051F824108A69694690477CBD00001E
:109FF0006D6F64756C6520726563762063616C6C4F
:10A000006261636B206572726F72210A000000004A
:10A010008C12002070B504460D460E490EA0F9F7CB
:10A0200035FC2E46601C18B911A0F9F72FFC10E082
:10A03000154850F8240060B1134850F82400C06956
:10A0400038B1114951F8240051F82410CA69314639
:10A05000904770BD65A6000825732C64656275671E
:10A060003A6E65745F746370206F6B0A00000000C5
:10A070006D6F64756C652063616C6C6261636B20ED
:10A080006572726F72210A008C12002038B5044686
:10A0900000BF1648C06940F002001449C861084674
:10A0A000C06900F00200009000BF00BF0622052139
:10A0B0001C20F6F7B8FF1C20F6F7A8FF4FF08040F1
:10A0C0000B49086048F69F404860002108488160BD
:10A0D00020884000401E0649C860002104480161F4
:10A0E000F7F789FB00F00EF838BD000000100240C1
:10A0F000B412002010B50248F7F7AEFB10BD000007
:10A10000B412002010B50248F7F7B5FB10BD0000EF
:10A11000B4120020F8B504460D46164617480570DF
:10A120001748066000BF1748C06940F00200154993
:10A13000C8610846C06900F00200009000BF00BF7F
:10A14000032211461D20F6F76EFF1D20F6F75EFF75
:10A150000D480E49086048F69F40486000210B48B2
:10A1600081606000401E0949C86000210748016104
:10A17000F7F741FB00F014F8F8BD000024000020C0
:10A180002800002000100240000400408405002048
:10A1900010B50248F7F760FB10BD000084050020F1
:10A1A00010B50248F7F767FB10BD000084050020DA
:10A1B00008B500BF1648C06940F004001449C861E2
:10A1C0000846C06900F00400009000BF00BF0622EE
:10A1D00005211E20F6F727FF1E20F6F717FF0D4872
:10A1E0000D49086048F69F40486000210A48816098
:10A1F0000A48006800884000401E0749C8600021E6
:10A2000005480161F7F7F7FA00F012F808BD000001
:10A210000010024000080040F4120020B0010020AD
:10A2200010B50248F7F718FB10BD0000F41200202B
:10A2300010B50248F7F71FFB10BD0000F412002014
:10A2400010B50446F8F732FC114812490860084678
:10A25000446000218160C16001610C2141610021E5
:10A260008161F7F709FC18B163210BA0F9F70CFB2A
:10A2700008480068C06840F0100006490968C860D6
:10A280004FF4FA720A490348F7F732FD10BD000097
:10A29000004400407C0400202E2E5C53595354454A
:10A2A0004D5C55736172745C75736172742E6300DA
:10A2B000C001002010B5044609480A490860084654
:10A2C000446000218160C160016181610C214161B4
:10A2D000F7F7D2FB012204490248F7F76BFD10BDE6
:10A2E00000480040BC0400201800002070B505465E
:10A2F0000C460120F9F7BCFA9620FAF73FFD2146FB
:10A3000005A0F9F7C3FA9620FAF738FD0020F9F70F
:10A31000AFFA002070BD00007572632068616E6442
:10A320006C65723A2025730A0000000038B50546B6
:10A3300000240020009000BF11E00B4A52F83410B6
:10A340002868F5F754FF40B9074800EBC4002968B6
:10A35000426868469047002038BD601CC4B2082C93
:10A36000EBD34FF0FF30F7E7100100202DE9FF4756
:10A3700006460D460027B8460620FCF7BBFA044601
:10A380008CB90120F9F774FA9620FAF7F7FC3249F4
:10A3900032A0F9F77BFA9620FAF7F0FC0020F9F7E3
:10A3A00067FABDE8FF872846FCF7A4FAC4F8020064
:10A3B000D4F8020098B90120F9F75AFA9620FAF772
:10A3C000DDFC254925A0F9F761FA9620FAF7D6FCBD
:10A3D0000020F9F74DFA2046FAF720FEE1E7D4F81D
:10A3E00002002A463146F5F7ADFE258002A9204637
:10A3F000FAF7C0FE8146BDF80A004FF6FB718842AD
:10A4000018D10120F9F734FA9620FAF7B7FC18A012
:10A41000F9F73CFA9620FAF7B1FC0020F9F728FA90
:10A420004846FAF79BFECDE9000108216846FFF790
:10A4300013FC00BFD4F8020030B1D4F80200FAF7E0
:10A44000EDFD0020C4F802001CB12046FAF7E6FD3D
:10A45000002400BFA5E7000020A6000825733A6D80
:10A46000616C6C6F63206572726F72210A0000006C
:10A4700050414E444F3A2073796E6368726F6E6933
:10A480007A652074696D650A000000000003030608
:10A4900001040602050003051F1C1F1E1F1E1F1FAF
:10A4A0001E1F1E1FA4A8000814A90008C8A70008A2
:10A4B000A4A8000814A900086CA70008A4A8000814
:10A4C00014A9000874A70008A4A8000814A900088B
:10A4D0007CA7000888A70008A4A8000814A9000801
:10A4E00078A80008A4A8000814A90008A4A80008D7
:10A4F00014A9000860A70008A4A8000814A900086F
:10A5000054A7000888A7000894A7000814A9000809
:10A51000A4A8000848A7000814A9000804A8000877
:10A52000A4A80008F8A70008B4A80008A4A8000878
:10A5300014A9000854A9000804A80008A4A8000849
:10A5400014A90008D8A7000834A7000840A90008EB
:10A55000A4A7000814A90008B8A70008000000007C
:10A5600000000000010203040607080900000000C3
:10A570000102030470616E646F5F7075626C6973D1
:10A58000685F646174615F6368616E6E656C310001
:10A590004900000000000000220000000000000050
:10A5A00022000000F8A90008D0A90008000000005F
:10A5B000E8A9000800000000DCA900080000000075
:10A5C0007B030000000000002200000038AA000801
:10A5D000220000000000000049000000010000000F
:10A5E0002200000000AA00082200000008AA0008BB
:10A5F00084AA00080000000010AA00080000000063
:10A600002CAA0008000000001CAA0008000000009E
:10A610007CAA0008000000007B050000000000008C
:10A620007A65726F5F6465766963655F64617461A2
:10A630005F70726F63657373006D7174745F7469BA
:10A640006D6572004D5154545F5461736B007463B7
:10A65000705F636F6E6E65637465645F63616C6C7D
:10A660006261636B007463705F73656E745F6361D6
:10A670006C6C6261636B007463705F646973636FB9
:10A680006E6E65637465645F63616C6C6261636B5D
:10A69000006E65745F7463705F73656E64000000C4
:10A6A0000100000045660008E566000800404040E3
:10A6B0004040404040404141414141404040404095
:10A6C0004040404040404040404040404005020241
:10A6D0000202020202020202020202020220202000
:10A6E000202020202020200202020202020290905C
:10A6F000909090901010101010101010101010105A
:10A7000010101010101010100202020202028888AD
:10A7100088888888080808080808080808080808B9
:10A7200008080808080808080202020240000000A1
:10A73000ADA600082B4343485F504545525F434C4C
:10A740004F5345443A2000002B43495053454E4453
:10A750003A2000002B4E4554434C4F53453A2000BD
:10A760002B4E45544F50454E3A2000002B43504944
:10A770004E3A20002B4353513A2000002B495041C0
:10A780004444523A200000002B4950204552524F79
:10A79000523A20002B4349504F50454E3A20312C1D
:10A7A000000000002B43485454504143543A204485
:10A7B0004154412C000000002B4348545450414365
:10A7C000543A2030000000002B4343485354415278
:10A7D000543A2030000000002B43434853454E4478
:10A7E0003A0000002B4950434C4F53453A000000BB
:10A7F0002B5354494E3A00002B4349504552524F77
:10A80000523A00003E00000041542B435053493F50
:10A810000000000041542B494643000041542B43A3
:10A82000434853454E44000041542B43495053453F
:10A830004E44000041542B4349504D4F44450000C5
:10A84000504220444F4E4500534D5320444F4E45F7
:10A850000000000041542B434348434C4F534500F4
:10A8600041542B434950434C4F53450041542B4EC8
:10A870004554434C4F5345004154450041542B43EC
:10A88000524547004F504C205550444154494E4783
:10A8900000000000504E4E205550444154494E4750
:10A8A000000000004F4B000041542B4343484F50E1
:10A8B000454E00002B4343484F50454E00000000DA
:10A8C00041542B4349504F50454E000041542B4EAC
:10A8D00045544F50454E000041542B4350494E00C3
:10A8E00041542B4347534E0041542B43495053523C
:10A8F0004950000041542B43434853544F500000EB
:10A9000041542B435351000041542B49504144447E
:10A91000520000004552524F5200000041542B4358
:10A92000485454504143540041542B4343485345E9
:10A930005400000041542B434348535441525400A7
:10A940002B43485454504143543A205245515545A5
:10A95000535400002B434348524543560000000027
:10A960002B4350494E3A20524541445900000000C3
:10A9700052445900504F535420257320485454508A
:10A980002F312E310D0A486F73743A2025733A2502
:10A99000640D0A4163636570743A2A2F2A0D0A43D5
:10A9A0006F6E6E656374696F6E3A20636C6F73656A
:10A9B0000D0A557365722D4167656E743A205349CF
:10A9C0004D373630300D0A25730D0A25730000000F
:10A9D0006465766963655F696400000070726F7416
:10A9E0006F636F6C000000006465766963655F7378
:10A9F00065637265740000006D717474000000007E
:10AA000053494D3736303000302E302E31000000A3
:10AA10006465766963655F636F6465006465766924
:10AA200063655F6D6F64756C6500000064657669D1
:10AA300063655F74797065003435343863636539F4
:10AA40003565653330393762343334613134353507
:10AA500034343565313038623637623430633065CE
:10AA600033383531306239393232356230646463BB
:10AA700065613630353438660000000076657273E3
:10AA8000696F6E0070726F647563745F6B657900D7
:10AA9000636C69656E742D3E636F6E6E7374617462
:10AAA000653A25642C20747970653A25642C205110
:10AAB0006F733A25642C2069643A25642C206D65F7
:10AAC0007373616765206C656E6774683A25640A04
:10AAD00000000000F4AA000800000020C0010000EF
:10AAE00032050008A8AB0008C0010020783500003E
:10AAF000EC3800084132100247011378A814081DF1
:10AB0000431B081408139D422B08D8101249120841
:10AB100012A91408A94A1B08E0101371545B0834E9
:10AB2000201ACC081311881B086C081355875B0882
:10AB30007C186A0808193813B9531B081C081391AC
:10AB40005B1B08C01813C19D1B0828081309605B14
:10AB50000860285AE8086910295029081A28382955
:10AB6000085A34081AA8181B5D445019081AD90845
:10AB70005A54285AF40813E4A71C08059F481930B2
:10AB800013EDA21B08F01029085A70101A84282906
:10AB9000085A94085A48085A4008F3FF01042CA2A6
:08ABA0004A041AFF01012C0018
:04000005080000ED02
:00000001FF
